:10631000E5467006127A8A8F4622E546B4050612D3
:106320003B478F4622E546B40B061270908F4622FB
:10633000E546B40A061267DD8F4622E546B40F062D
:10634000126FFC8F4622E546B414061260E28F46B7
:1063500022E546B41906127A158F4622E546B41E88
:1063600006127A9E8F4622E546B42306126B8E8F64
:106370004622E546B42806127B538F4622E546B4F2
:106380002D06127AB28F4622E546B432051272EF1C
:036390008F462213
:107A8A00C20890061EE0FFA3E0901CECCFF0A3EF23
:047A9A00F07F052252
:103B4700127B4F50477D047F011262885008E53E83
:103B5700B401037F0B227D047F021262885008E5BF
:103B67003EB402037F0B227D047F03126288500854
:103B7700E53EB403037F0B227D047F041262885065
:103B870008E53EB404037F0B227F0A227F081274E4
:103B9700D650061253027F00227D057F05126288E8
:103BA7005032901CEEE07002A3E070282046257D7D
:103BB700017F011262884003023CBD90066CE0FF62
:103BC7007C0A7D70127234900610E0FFA3E0901C0F
:103BD700EE023C847D067F051262885031901CF00E
:103BE700E07002A3E070272048247D017F02126263
:103BF700884003023CBD90066DE0FF7C0A7D901271
:103C07007234900612E0FFA3E0901CF0806F7D07EE
:103C17007F051262885031901CF2E07002A3E070B9
:103C270027204C247D017F031262884003023CBD9C
:103C370090066EE0FF7C0A7DB0127234900614E0A5
:103C4700FFA3E0901CF280357D087F051262885043
:103C570033901CF4E07002A3E07029204F267D0109
:103C67007F04126288504F90066FE0FF7C0A7DD078
:103C7700127234900616E0FFA3E0901CF4CFF0A375
:103C8700EFF080327D077F06126288500F30290CD3
:103C9700901CECE07002A3E07002C22930380C904F
:103CA7001CECE07002A3E07002C238786CE6B40541
:093CB700057F041260507F052214
:10709000203842900633E0901D10F012331EE53E7A
:1070A000B401062049247F0522E53EB40206204DA6
:1070B000197F0522E53EB4030620510E7F0522E527
:1070C0003EB404062054037F0522901D10E0D394A3
:0870D0000050C8D2387F0A22EB
:1067DD00E53B700AE53EB40105753B018028E53BBC
:1067ED00700AE53EB40205753B02801AE53B700A5E
:1067FD00E53EB40305753B03800CE53B7008E53EB3
:10680D00B40403753B047D077F06126288500C7D2E
:10681D00077F06126288501E30291B900650E0FF3C
:10682D007C067DF01272347D017F01126288500664
:09683D00120FB3122B3C7F0F2255
:106FFC00127B4F503F120FB3202F09203006203147
:10700C0003303209E53270051276CB800B786CE6D2
:10701C00B4050B7F03126050122B3C120FB3202FC0
:10702C001020300D20310A203207E5327003122B6C
:0A703C003C7F0F221276CB7F142256
:1060E200E4F53B900651E0FF7C077D101272347D8F
:1060F200077F06126288500C7D077F061262885065
:106102005E30295B786CE670047F018008786CE66B
:10611200B404077F021260508038786CE6B407043A
:106122007601802E7D037F051262885025901CF631
:10613200E07002A3E0701B900662E0FF7C097D30F4
:10614200127234900620E0FFA3E0901CF6CFF0A379
:10615200EFF07F061274D650037F00227F19227D52
:0E616200077F0612628850052029027F052261
:107A15007D077F0612628850062029037F05229084
:0A7A25000630E0901D10F07F1E22D5
:107A9E00901D10E070037F2322127B4F50037F0A4C
:047AAE00227F1E22F3
:106B8E007D047F071262885041E53EB4010B9006EA
:106B9E005EE0FF7C087DB0802EE53EB4020B9006D1
:106BAE005FE0FF7C087DD0801EE53EB4030B9006AF
:106BBE0060E0FF7C087DF0800EE53EB4040C90068C
:106BCE0061E0FF7C097D10127234900631E0901D59
:056BDE0010F07F2822E9
:037B53007F2D2261
:107AB200901D10E070037F3222127B4F50037F0A29
:047AC200227F2D22D0
:1072EF003058037F32227D047F0512628850289028
:1072FF001CF8E07002A3E0701E900663E0FF7C09AB
:10730F007D50127234900622E0FFA3E0901CF8CF5C
:0C731F00F0A3EFF07F3222C2087F0022B2
:10736400D224753D0312331E122B3C120FB3127B31
:107374004F5009E53D600512331E80F2E4F522F515
:1073840023127B4F4009E53D600512331E80F2E570
:087394003D70D2C224C2582250
:04000E0001000130BC
:0300030002690E81
:0B690E00C0E0C083C082C0D075D0087C
:10691900853082852F83E493FF204404C4540FFFFC
:10692900430FF08F80C284D28500C2870000D287CE
:10693900007580FF7580FEC284C28500C287000091
:106949000000D287007580FF30440CC2440530E551
:0B695900307006052F8002D244D2A847
:09696400D0D0D082D083D0E03203
:03000B00021BB61F
:101BB600C0E0C0F0C083C082C0D075D008758CD894
:101BC600758A92D28C1241ED12743BE531D39400A2
:101BD60040051531021F40753111901D10E0D39458
:101BE600004003E014F0901D11E0D394004003E0A0
:101BF60014F0901D12E0D394004003E014F0901D01
:101C060013E0D394004003E014F0E532D39400408F
:101C16000215321541E541B40A004003021F3D900A
:101C26001C2CF8282873021F40021E91021E59021E
:101C36001E2C021DC2021D58021CEE021C84021C30
:101C460067021C4AD3901CEDE09400901CECE094D3
:101C5600005003021F40A3E024FFF0901CEC021F7B
:101C660031D3901CE9E09400901CE8E09400500306
:101C7600021F40A3E024FFF0901CE8021F317F0101
:101C86001277934003021F40901CE1E09400901CE1
:101C9600E0E09400400CA3E024FFF0901CE0E03468
:101CA600FFF0D3901CEFE09400901CEEE09400400F
:101CB6000CA3E024FFF0901CEEE034FFF0D3901C60
:101CC600FBE09400901CFAE094005003021F407D54
:101CD600067F011262884003021F40901CFBE0242D
:101CE600FFF0901CFA021F317F0212779340030225
:101CF6001F40901CE3E09400901CE2E09400400C2E
:101D0600A3E024FFF0901CE2E034FFF0D3901CF136
:101D1600E09400901CF0E09400400CA3E024FFF057
:101D2600901CF0E034FFF0D3901CFDE09400901C72
:101D3600FCE094005003021F407D067F0212628879
:101D46004003021F40901CFDE024FFF0901CFC02A3
:101D56001F317F031277934003021F40901CE5E07A
:101D66009400901CE4E09400400CA3E024FFF09063
:101D76001CE4E034FFF0D3901CF3E09400901CF2D6
:101D8600E09400400CA3E024FFF0901CF2E034FF46
:101D9600F0D3901CFFE09400901CFEE094005003EA
:101DA600021F407D067F031262884003021F409097
:101DB6001CFFE024FFF0901CFE021F317F04127707
:101DC600934003021F40901CE7E09400901CE6E05D
:101DD6009400400CA3E024FFF0901CE6E034FFF0F2
:101DE600D3901CF5E09400901CF4E09400400CA302
:101DF600E024FFF0901CF4E034FFF0D3901D01E0E6
:101E06009400901D00E094005003021F407D067F61
:101E1600041262884003021F40901D01E024FFF077
:101E2600901D00021F31D3901CEBE09400901CEA39
:101E3600E09400400CA3E024FFF0901CEAE034FF9D
:101E4600F0901D14E0D394005003021F40E014F0FC
:101E5600021F40D3901CF9E09400901CF8E0940017
:101E6600400CA3E024FFF0901CF8E034FFF0D39080
:101E76001CF7E09400901CF6E094005003021F400B
:101E8600A3E024FFF0901CF6021F31786CE6FF7089
:101E960003021F40EFB401059006188027786CE610
:101EA600FFB40219D3901CEBE09400901CEAE09476
:101EB60000403FA3E024FFF0901CEA806EEFB403DD
:101EC6001190061AE0FFA3E0901CEACFF0A3EFF012
:101ED6008020786CE6FFB4041ED3901CEBE09400DF
:101EE600901CEAE09400400AA3E024FFF0901CEA6C
:101EF6008039786C068043EF6405603E786CE6FFB7
:101F0600B4060D901CEA7402F0A37458F006802AF9
:101F1600EFB40726D3901CEBE09400901CEAE09403
:101F260000400EA3E024FFF0901CEAE034FFF080AE
:101F360009786C7600800375410A1279C24008124E
:101F4600759940031279DED0D0D082D083D0F0D0FC
:021F5600E03277
:0300130002617017
:0D617000C0E0C0F0C083C082C0D075D01068
:10617D0075A0FFC284C285D287C286308018C2A4A2
:10618D00C2A5D2A6C2A7E5A0540FF54AD2A7FF1209
:10619D00660DD286804F308118D2A4C2A5D2A6C278
:1061AD00A7E5A0540FF54AD2A7FF126393D28680BC
:1061BD0034308218C2A4D2A5D2A6C2A7E5A0540F2E
:1061CD00F54AD2A7FF126413D2868019308316D2F6
:1061DD00A4D2A5D2A6C2A7E5A0540FF54AD2A7FF17
:0561ED00126493D2864C
:0B61F200D0D0D082D083D0F0D0E032BB
:106B3700BF0113900632E0901D10F0901D10E0D3B6
:106B47009400404280F5BF0213900632E0901D1179
:106B5700F0901D11E0D39400402C80F5BF031390F3
:106B67000632E0901D12F0901D12E0D394004016FB
:106B770080F5BF0411900632E0901D13F0901D13AD
:076B8700E0D3940050F72257
:106BE300304712205D0F900672E0FF7C0B7D301260
:106BF3007234D25D22304B12205F0F900673E0FF98
:106C03007C0B7D50127234D25F22304E1220600F03
:106C1300900674E0FF7C0B7D70127234D2602230D8
:106C2300521120610E900675E0FF7C0B7D9012726D
:046C330034D26122D4
:10558200303D1A204617900664E0FF7C097D7012B8
:105592007234D246C214C210C21CC218223046143F
:1055A200203911900665E0FF7C097D90127234C2A9
:1055B20046C23D22303E1A204817900666E0FF7C24
:1055C200097DB0127234D248C215C211C21DC2196D
:1055D20022304814203A11900667E0FF7C097DD002
:1055E200127234C248C23E2230401A204C17900632
:1055F20068E0FF7C097DF0127234D24CC216C212EE
:10560200C21EC21A22304C14203B11900669E0FFE0
:105612007C0A7D10127234C24CC2402230421A20DF
:105622004F1790066AE0FF7C0A7D30127234D24F27
:10563200C217C213C21FC21B22304F13203C10904C
:10564200066BE0FF7C0A7D50127234C24FC24222C6
:10514B001240D3D28C7F071274D6500512001680F2
:10515B00121271207F1F7E001277E090001FEFF07C
:10516B001275F37F081274D6500512594A80FE90BF
:10517B0006087402F0A37458F090060A7402F0A3A8
:10518B007458F090060C7402F0A37458F090060E4D
:10519B007402F0A37458F0900681E0FF7C0D7D1033
:1051AB00127234E4FFEFFD3395E0FC74302DF58281
:1051BB0074003CF583E0FE74F02DF582741A3CF517
:1051CB0083EEF00FBF08DED2081279DE7545017F42
:1051DB0001126050900618E0FFA3E0901CEACFF09C
:1051EB00A3EFF0C2081279DE12331E12631030598E
:1051FB0003124418305A03124305305B0312485B09
:10520B00305E03124965124D747D077F061262886A
:0C521B004002C229125582126BE380CCC5
:104418007C007D80C2657F0112368D50117F0612A7
:1044280074D65002D2087F01121F580244B87C008B
:104438007D70D2657F0112368D5002800D7C007D23
:1044480078D2657F0112368D50077F0112094180AD
:104458005F7C007DA0D2657F0112368D50117D07EB
:104468007F0612628850087545011276F480417CF7
:10447800007DA8C2657F0112368D50197D057F0128
:1044880012628850107F061274D65002D2087F013B
:1044980012452A801B7C007DB0C2657F0112368DD3
:1044A800500E7F061274D65002D2087F01124F6454
:1044B800E4F54CAF4CEF3395E0FEEF7803C333CE11
:1044C80033CED8F92400F58274013EAD82FCD26562
:1044D8007F0112368D5038754501AF4CEF3395E0AA
:1044E800FE74A02FF58274063EF583E0FFC007AF87
:1044F8004CEF3395E0FEEF7805C333CE33CED8F9D1
:1045080024F0F58274103EAD82FCD007126E2C05A3
:104518004CC3E54C648094A84099C259C263126C9C
:01452800375B
:01452900226F
:104305007F061274D65002C2087D017F06126288AC
:10431500503D7C007D88C2657F0212368D500BD2E0
:10432500097F02121F58C20980257C007D70D26565
:104335007F0212368D5002800D7C007D78D2657F1C
:104345000212368D5009D2097F02120941C2099025
:10435500001FE030E1427C007DA0D2657F0212366D
:104365008D50147D077F06126288500B12780675F2
:1043750045021276F4801E7C007DA8C2657F02127C
:10438500368D50147D057F02126288500B12780617
:104395007F0212452A1278D67D027F061262885066
:1043A5006AE4F54CAF4CEF3395E0FEEF7803C33389
:1043B500CE33CED8F92400F58274013EAD82FCD20D
:1043C500657F0212368D5038754502AF4CEF339537
:1043D500E0FE74A02FF58274063EF583E0FFC0076A
:1043E500AF4CEF3395E0FEEF7805C333CE33CED82F
:1043F500F924F0F58274103EAD82FCD007126E2CC4
:10440500054CC3E54C648094A84099C25AC2641215
:024415006C8BAE
:014417002282
:10485B007D037F06126288503D7C007D90C2657F90
:10486B000312368D500BD20E7F03121F58C20E80CF
:10487B00257C007D70D2657F0312368D5002800D32
:10488B007C007D78D2657F0312368D5009D20E7F66
:10489B0003120941C20E90001FE030E2427C007D02
:1048AB00A0D2657F0312368D50147D077F061262EE
:1048BB0088500B1278067545031276F4801E7C0027
:1048CB007DA8C2657F0312368D50147D057F0312C0
:1048DB006288500B1278067F0312452A1278D67D18
:1048EB00047F06126288506AE4F54CAF4CEF3395A7
:1048FB00E0FEEF7803C333CE33CED8F92400F58234
:10490B0074013EAD82FCD2657F0312368D50387533
:10491B004503AF4CEF3395E0FE74A02FF582740680
:10492B003EF583E0FFC007AF4CEF3395E0FEEF7829
:10493B0005C333CE33CED8F924F0F58274103EADD7
:10494B0082FCD007126E2C054CC3E54C648094A8F6
:09495B004099C25BC228126CDF16
:014964002230
:104965007D057F06126288503D7C007D98C2657F7B
:104975000412368D500BD20C7F04121F58C20C80C6
:10498500257C007D70D2657F0412368D5002800D26
:104995007C007D78D2657F0412368D5009D20C7F5C
:1049A50004120941C20C90001FE030E3427C007DF7
:1049B500A0D2657F0412368D50147D077F061262E2
:1049C50088500B1278067545041276F4801E7C001B
:1049D5007DA8C2657F0412368D50147D057F0412B3
:1049E5006288500B1278067F0412452A1278D67D0C
:1049F500067F06126288506AE4F54CAF4CEF33959A
:104A0500E0FEEF7803C333CE33CED8F92400F58228
:104A150074013EAD82FCD2657F0412368D50387527
:104A25004504AF4CEF3395E0FE74A02FF582740674
:104A35003EF583E0FFC007AF4CEF3395E0FEEF781E
:104A450005C333CE33CED8F924F0F58274103EADCC
:104A550082FCD007126E2C054CC3E54C648094A8EB
:094A65004099C25EC22A126D33B1
:014A6E002225
:106ECC00BF010AC214C210C21CC2188025BF020A1C
:106EDC00C215C211C21DC2198018BF030AC216C244
:106EEC0012C21EC21A800BBF0408C217C213C21FE3
:106EFC00C21B90001FE0FF30E002D224EF30E10211
:0E6F0C00D225EF30E202D226EF30E302D22788
:016F1A002254
:10660D008F4B7868E6C39450506E30496B7D077F91
:10661D0001126288502B205C287868E6700D900678
:10662D003BE0B54B06203F03D23F22202F0D203FEC
:10663D000A7F01126ECC753D02D22F900634E0F523
:10664D00327D087F06126288501990063FE0B54BE7
:10665D0006205C03D263220534E534AE33700E059B
:10666D0033800A0534E534AE337002053314F582F8
:09667D008E83E54BF078680622DB
:106393008F4B7869E6C394505075304D727D077FFB
:1063A3000212628850327F02127793502B205C28AE
:1063B3007869E6700D90063BE0B54B06204103D2A9
:1063C300412220300D20410A7F02126ECC753D021E
:1063D300D230900634E0F5327D087F061262885091
:1063E3001990063FE0B54B06205C03D264220536C4
:1063F300E536AE35700E0535800A0536E536AE3521
:106403007002053514F5828E83E54BF07869062218
:106413008F4B786AE6C3945050753051727D077F75
:106423000312628850327F03127793502B205C282B
:10643300786AE6700D90063BE0B54B06204303D225
:10644300432220310D20430A7F03126ECC753D0297
:10645300D231900634E0F5327D087F06126288500F
:106463001990063FE0B54B06205C03D2282205387D
:10647300E538AE37700E0537800A0538E538AE3794
:106483007002053714F5828E83E54BF0786A062295
:106493008F4B786BE6C3945050753054727D077FF1
:1064A3000412628850327F04127793502B205C28A9
:1064B300786BE6700D90063BE0B54B06204503D2A2
:1064C300452220320D20450A7F04126ECC753D0211
:1064D300D232900634E0F5327D087F06126288508E
:1064E3001990063FE0B54B06205C03D22A22053AF9
:1064F300E53AAE39700E0539800A053AE53AAE3908
:106503007002053914F5828E83E54BF0786B062211
:1078060090001FE0FF30E004D208D220EF30E10400
:10781600D209D221EF30E204D20ED222EF30E304B5
:05782600D20CD2232268
:1078D600C220C221C222C22390001FE0FF30E10273
:0F78E600C209EF30E202C20EEF30E302C20C2201
:106050008F4C3046030260DD3048030260DD204C87
:106060007C204F79E54CB401197D017F05126288CF
:10607000500C90065AE0FF7C087D30127234786C28
:106080000622E54CB402177D027F05126288504853
:1060900090065BE0FF7C087D50127234803AE54C3C
:1060A000B4041A7D027F05126288500C90065DE0F0
:1060B000FF7C087D90127234786C760622E54C6481
:1060C00003701E7D027F05126288500C90065CE012
:1060D000FF7C087D70127234786C760122E4786C53
:0260E000F622A6
:1079FA00EF1FAA0670011ED39400EA9400400BE41C
:0A7A0A00FDEDC394C850E90D80F7AC
:017A1400224F
:1059FF008F5D30695BE55DB40111D22090001FE02F
:105A0F00F420E003305C44D2088040E55DB402111D
:105A1F00D22190001FE0F420E103305C2ED20980E8
:105A2F002AE55DB40311D22290001FE0F420E203B7
:105A3F00305C18D20E8014E55DB4040FD2239000B1
:105A4F001FE0F420E303305C02D20CAF5D026B3732
:105A5F00E55DB40110C22090001FE0F420E0033098
:105A6F005C41C20822E55DB40210C22190001FE024
:105A7F00F420E103305C2CC20922E55DB40310C2AF
:105A8F002290001FE0F420E203305C17C20E22E5E3
:105A9F005DB4040FC22390001FE0F420E303305CD9
:045AAF0002C20C2201
:105AB3008F5330675BE553B40111D22490001FE08C
:105AC300F420E003305C44D2088040E553B4021173
:105AD300D22590001FE0F420E103305C2ED2098030
:105AE3002AE553B40311D22690001FE0F420E20309
:105AF300305C18D20E8014E553B4040FD227900003
:105B03001FE0F420E303305C02D20CAF53026B3787
:105B1300E553B40110C22490001FE0F420E00330E9
:105B23005C41C20822E553B40210C22590001FE075
:105B3300F420E103305C2CC20922E553B40310C204
:105B43002690001FE0F420E203305C17C20E22E52A
:105B530053B4040FC22790001FE0F420E303305C2A
:045B630002C20C224C
:0828E6008F538C548D558B5665
:1028EE00C265E55524FFF582E55434FFF583E0F526
:1028FE0058855582855483E0FFF559A3E0FEF55ABD
:10290E00EF14B40800505C90292375F003A4C5831E
:10291E0025F0C5837302293B022942022949022967
:10292E005002295702295E02296502296C7557014A
:10293E00D265802F755702D2658028755704D265EF
:10294E008021755708D265801A755710D26580138D
:10295E00755720D265800C755740D2658005755726
:10296E0080D265EE24FE7003022A3324F8605C24C4
:10297E00096003022A45E553B40105900020804505
:10298E00E553B40205900021803BE553B403059056
:10299E0000228031E553B404059000238027E553CF
:1029AE00B40505900024801DE553B406059000255E
:1029BE008013E553B407059000268009E55364089B
:1029CE007077900027E04557F0806EE553B401050F
:1029DE009000208045E553B40205900021803BE530
:1029EE0053B403059000228031E553B404059000E2
:1029FE00238027E553B40505900024801DE553B4CC
:102A0E0006059000258013E553B407059000268037
:102A1E0009E55364087022900027E0FFE557F4FEA5
:102A2E00EF5EF08014E553B4080D8555828554830E
:102A3E00E0FF125FBCC265C265206503022B3BE559
:102A4E0053B40109900020E0FD7F208060E553B46F
:102A5E000209900021E0FD7F218052E553B4030965
:102A6E00900022E0FD7F228044E553B404099000DB
:102A7E0023E0FD7F238036E553B40509900024E062
:102A8E00FD7F248028E553B40609900025E0FD7FE4
:102A9E0025801AE553B40709900026E0FD7F2680B5
:102AAE000CE553B4080C900027E0FD7F277E001242
:102ABE007274D2AFD269AF561259FFAD58E4FF12FD
:102ACE007677AD59E4FF127677E55AB401047D3876
:102ADE008007E55AB40A077D367F06127677E553EE
:102AEE00B408031275F37D077F06126288500B201F
:102AFE002908C208C209C20EC20C7D017F011262F2
:102B0E00884002C2087D017F021262884002C2091B
:102B1E007D017F031262884002C20E7D017F041286
:0D2B2E0062884002C20CC269AF561259FF06
:012B3B002277
:045D55008F538D5487
:105D5900D269AF541259FFAF54126B37E553B401EE
:105D6900059000208044E553B40205900021803A53
:105D7900E553B403059000228030E553B40405903F
:105D890000238026E553B40505900024801CE553C3
:105D9900B406059000258012E553B4070590002646
:105DA9008008E553B40806900027E0F555E55560ED
:105DB90025755701E4F556E55530E007AD57E4FF81
:105DC900127677E555C313F55505570556E556C3BC
:105DD900940840E3800E7D187F021276777D537F09
:0B5DE90002127677C269AF541259FF16
:015DF400228C
:021F58008F4DAB
:101F5A00E54D6401701E754E1B754F10900080E0B0
:101F6A00F550E54F2550F582E4354EF583E0F552FC
:101F7A0078688069E54D6402701E754E1B754F6066
:101F8A00900088E0F550E54F2550F582E4354EF58E
:101F9A0083E0F55278698045E54D6403701E754EFD
:101FAA001B754FB0900090E0F550E54F2550F58233
:101FBA00E4354EF583E0F552786A8021E54DB404A4
:101FCA001F754E1C754F00900098E0F550E54F259F
:101FDA0050F582E4354EF583E0F552786BE6F5511B
:101FEA00E55214B4090040030222F790200375F069
:101FFA0003A4C58325F0C5837302201E0220710243
:10200A0020C402211702216A0221BD0222100222E3
:10201A00610222B1E54F2550F582E4354EF583A3DE
:10202A00E0B40A18E5502402FFE433FEE551B5078F
:10203A000BE4B50607AD4D7F01022286AF507E0044
:10204A00EF2403FDEE33FCE5516D7001EC600302F1
:10205A0022F7EF254FFFEE354ECF2401FDE43FFC7A
:10206A00AB4D7F010222AEE54F2550F582E4354E95
:10207A00F583A3E0B40A18E5502402FFE433FEE531
:10208A0051B5070BE4B50607AD4D7F02022286AFB4
:10209A00507E00EF2403FDEE33FCE5516D7001EC38
:1020AA0060030222F7EF254FFFEE354ECF2401FDE4
:1020BA00E43FFCAB4D7F020222AEE54F2550F5828C
:1020CA00E4354EF583A3E0B40A18E5502402FFE490
:1020DA0033FEE551B5070BE4B50607AD4D7F0302A4
:1020EA002286AF507E00EF2403FDEE33FCE5516DEE
:1020FA007001EC60030222F7EF254FFFEE354ECF59
:10210A002401FDE43FFCAB4D7F030222AEE54F25DF
:10211A0050F582E4354EF583A3E0B40A18E550245D
:10212A0002FFE433FEE551B5070BE4B50607AD4DF2
:10213A007F04022286AF507E00EF2403FDEE33FCBB
:10214A00E5516D7001EC60030222F7EF254FFFEEB7
:10215A00354ECF2401FDE43FFCAB4D7F040222AE95
:10216A00E54F2550F582E4354EF583A3E0B40A180D
:10217A00E5502402FFE433FEE551B5070BE4B5064A
:10218A0007AD4D7F05022286AF507E00EF2403FD86
:10219A00EE33FCE5516D7001EC60030222F7EF2586
:1021AA004FFFEE354ECF2401FDE43FFCAB4D7F05DA
:1021BA000222AEE54F2550F582E4354EF583A3E0C1
:1021CA00B40A18E5502402FFE433FEE551B5070BC3
:1021DA00E4B50607AD4D7F06022286AF507E00EFBA
:1021EA002403FDEE33FCE5516D7001EC600302221D
:1021FA00F7EF254FFFEE354ECF2401FDE43FFCAB50
:10220A004D7F060222AEE54F2550F582E4354EF5A4
:10221A0083A3E0B40A17E5502402FFE433FEE55134
:10222A00B5070AE4B50606AD4D7F07804FAF507E6D
:10223A0000EF2403FDEE33FCE5516D7001EC600301
:10224A000222F7EF254FFFEE354ECF2401FDE43F82
:10225A00FCAB4D7F07804DE54F2550F582E4354EA6
:10226A00F583A3E0B40A18E5502402FFE433FEE53F
:10227A0051B5070BE4B50607AD4D7F08025D55AFB2
:10228A00507E00EF2403FDEE33FCE5516D7001EC46
:10229A00705BEF254FFFEE354ECF2401FDE43FFC86
:1022AA00AB4D7F080228E6E54F2550F582E4354E0E
:1022BA00F583A3A3E07036E54F2550F582E4354E49
:1022CA00F583A3E024F96008147022AF4D02776CFD
:1022DA00D2697F011259FFAF4D126B377D5E7F02C3
:0D22EA00127677C2697F011259FF12594A1E
:0122F70022C4
:04368D008C4D8D4E85
:10369100054EE54E7002054D14F5828C83E0F970FC
:1036A1000302382FBF010875331B753410801FBF0B
:1036B100020875351B7536608014BF030875371B0A
:1036C1007538B08009BF040675391C753A0020654C
:1036D10003023795BF01087868E6696002C322BF1B
:1036E10002087869E6696002C322BF0308786AE6C6
:1036F100696002C322BF0408786BE6696002C322D5
:10370100E4FEEEC3994003023793EF6401701CE5B8
:103711004E2EF582E4354DF583E0FDE5342EF5823C
:10372100E43533F583E06D6002C322EF6402701C5F
:10373100E54E2EF582E4354DF583E0FDE5362EF5B7
:1037410082E43535F583E06D6002C322EF640370D6
:103751001CE54E2EF582E4354DF583E0FDE5382E6E
:10376100F582E43537F583E06D6002C322EF64042E
:10377100701CE54E2EF582E4354DF583E0FDE53A0A
:103781002EF582E43539F583E06D6002C3220E0225
:103791003703D322306503023830E4FEEEC399408B
:1037A1000302382DEF6401701CE54E2EF582E435DD
:1037B1004DF583E0FDE5342EF582E43533F583E004
:1037C1006D6065C322EF6402701CE54E2EF582E444
:1037D100354DF583E0FDE5362EF582E43535F5838B
:1037E100E06D6044C322EF6403701CE54E2EF58248
:1037F100E4354DF583E0FDE5382EF582E43537F506
:1038010083E06D6023C322EF6404701CE54E2EF546
:1038110082E4354DF583E0FDE53A2EF582E4353954
:0F382100F583E06D6002C3220E02379DD322C3F0
:013830002275
:102B3C0090001FE0540FF55CB4010BE53EB40103AB
:102B4C00D21422C21422E55C6403702AE53EB4015F
:102B5C0006D214D2108004C214C210E53EB4021185
:102B6C00D2157D017F071262884003022D57D211C6
:102B7C0022C215C21122E55C6405702AE53EB4013F
:102B8C0006D214D21C8004C214C21CE53EB403113C
:102B9C00D2167D027F071262884003022D57D21E87
:102BAC0022C216C21E22E55C6409702AE53EB401FD
:102BBC0006D214D2188004C214C218E53EB4041113
:102BCC00D2177D037F071262884003022D57D21B58
:102BDC0022C217C21B22E55C6407704EE53EB401AD
:102BEC0008D214D210D21C8006C214C210C21CE52A
:102BFC003EB40211D2157D017F071262885002D2B9
:102C0C0011D21D8006C215C211C21DE53EB40313BC
:102C1C00D216D2127D027F071262884003022D5712
:102C2C00D21E22C216C212C21E22E55C640B704E6A
:102C3C00E53EB40108D214D210D2188006C214C2D8
:102C4C0010C218E53EB40211D2157D017F07126245
:102C5C00885002D211D2198006C215C211C219E5D0
:102C6C003EB40413D217D2137D037F07126288403F
:102C7C0003022D57D21B22C217C213C21B22E55CC2
:102C8C00640D704BE53EB40108D214D21CD21880EE
:102C9C0006C214C21CC218E53EB40311D2167D0242
:102CAC007F071262885002D21ED21A8006C216C248
:102CBC001EC21AE53EB40413D217D21F7D037F0740
:102CCC001262884003022D57D21B22C2178078E56E
:102CDC005C640F7076E53EB4010AD214D210D21C9B
:102CEC00D2188008C214C210C21CC218E53EB4022D
:102CFC0013D2157D017F071262885002D211D21DAA
:102D0C00D2198008C215C211C21DC219E53EB40306
:102D1C0013D216D2127D027F071262885002D21E85
:102D2C00D21A8008C216C212C21EC21AE53EB404E0
:102D3C0012D217D213D21F7D037F07126288500B59
:0B2D4C00D21B22C217C213C21FC21B01
:012D57002259
:100FB30090001FE0540FF55CB401167D017F011210
:100FC3006288500A7F061274D64003D20822C208F0
:100FD30022E55C6403705BE53E640170257D017F5F
:100FE30001126288500B7F061274D64004D2088027
:100FF30002C2087D017F021262885003D20922C215
:101003000922E53E640260030214637D017F01123D
:1010130062885004D2088002C2087D017F021262F6
:1010230088500C7D017F071262885003D20922C2C7
:101033000922E55C6405705BE53E640170257D0172
:101043007F01126288500B7F061274D64004D208C7
:101053008002C2087D017F031262885003D20E22F0
:10106300C20E22E53E640360030214637D017F0127
:101073001262885004D2088002C2087D017F0312E5
:101083006288500C7D027F071262885003D20E22C1
:10109300C20E22E55C6409705BE53E640170257D48
:1010A300017F01126288500B7F061274D64004D26E
:1010B300088002C2087D017F041262885003D20CAB
:1010C30022C20C22E53E640460030214637D017FA7
:1010D300011262885004D2088002C2087D017F0495
:1010E300126288500C7D037F071262885003D20C72
:1010F30022C20C22E55C640760030211B5E53E647D
:101103000170347D017F01126288500B7F061274D7
:10111300D64004D2088002C2087D017F0212628891
:101123005004D2098002C2097D017F0312628850F4
:1011330003D20E22C20E22E53E640270367D017F89
:10114300011262885004D2088002C2087D017F0226
:10115300126288500D7D017F071262885004D20904
:101163008002C2097D017F031262885003D20E22DE
:10117300C20E22E53E640360030214637D017F0116
:101183001262885004D2088002C2087D017F0212D5
:1011930062885004D2098002C2097D017F03126272
:1011A30088500C7D027F071262885003D20E22C240
:1011B3000E22E55C640B6003021273E53E6401706A
:1011C300347D017F01126288500B7F061274D64072
:1011D30004D2088002C2087D017F02126288500493
:1011E300D2098002C2097D017F041262885003D2B2
:1011F3000C22C20C22E53E640270367D017F01128F
:1012030062885004D2088002C2087D017F02126204
:1012130088500D7D017F071262885004D209800235
:10122300C2097D017F041262885003D20C22C20CD2
:1012330022E53E640460030214637D017F011262B0
:10124300885004D2088002C2087D017F021262889E
:101253005004D2098002C2097D017F0412628850C2
:101263000C7D037F071262885003D20C22C20C222A
:10127300E55C640D6003021331E53E640170347D67
:10128300017F01126288500B7F061274D64004D28C
:10129300088002C2087D017F031262885004D20EC7
:1012A3008002C20E7D017F041262885003D20C2299
:1012B300C20C22E53E640370367D017F0112628811
:1012C3005004D2088002C2087D017F031262885055
:1012D3000D7D027F071262885004D20E8002C20E77
:1012E3007D017F041262885003D20C22C20C22E5D6
:1012F3003E640460030214637D017F01126288501F
:1013030004D2088002C2087D017F03126288500460
:10131300D20E8002C20E7D017F04126288500C7DC2
:10132300037F071262885003D20C22C20C22E55CB1
:10133300640F6003021463E53E640170437D017F23
:1013430001126288500B7F061274D64004D20880C3
:1013530002C2087D017F021262885004D209800212
:10136300C2097D017F031262885004D20E8002C23B
:101373000E7D017F041262885003D20C22C20C221C
:10138300E53E640270457D017F011262885004D2FC
:10139300088002C2087D017F02126288500D7D0120
:1013A3007F071262885004D2098002C2097D017F3F
:1013B300031262885004D20E8002C20E7D017F04A4
:1013C3001262885003D20C22C20C22E53E640370E1
:1013D300457D017F011262885004D2088002C20851
:1013E3007D017F021262885004D2098002C2097D06
:1013F300017F03126288500D7D027F0712628850BD
:1014030004D20E8002C20E7D017F04126288500353
:10141300D20C22C20C22E53E640470447D017F019C
:101423001262885004D2088002C2087D017F021232
:1014330062885004D2098002C2097D017F031262CF
:10144300885004D20E8002C20E7D017F041262888E
:10145300500C7D037F071262885003D20C22C20C0A
:011463002266
:1077BA007F011277935015E53BB40110C209C20E3E
:1077CA00C20C7F061274D6500CC208227F011277AF
:0677DA00934002C20822E8
:107931007F02127793500CE53BB40207C209C20ED5
:0D794100C20C227F021277934002C209227D
:10794E007F03127793500CE53BB40307C209C20EB6
:0D795E00C20C227F031277934002C20E225A
:10796B007F04127793500CE53BB40407C209C20E97
:0D797B00C20C227F041277934002C20C223E
:10696D000500050105030507050F051F051E051C7F
:10697D00051805100201040E040A03060101040B9B
:10698D000304040F020304010302040D02000202BA
:10699D0003000409040403050307010003030407AE
:1069AD00030104060402040C051605150000061566
:0E69BD00062A060C06380633061E06120617BA
:10522700203737900640E004F519D3648094815005
:1052370003025301D3E5196480948F400375190F56
:1052470090063DE0FF123E3490063EE0F518E4F587
:105257001ED237C262C257C24A22304A6030621633
:10526700152EE52ED394004003025301C2CAC26231
:10527700D25785182E2230570E152EE52ED39400BF
:105287005078C262C25722AF1C151CEF700BC24A7E
:10529700E51825E0F52ED25722E51D30E0058518E3
:1052A7002E8008E51875F003A4F52EAF1D7801EFE1
:1052B70008800103D8FDF51DD262D2CA22D519088C
:1052C700C237E4F53DC25822051E7440251EF582FB
:1052D700E43406F583E025E0246DF582E43469F5CE
:1052E70083E493540FF51C740193F51D700AD2578C
:0A52F700E51825E025E0F52ED24A67
:015301002289
:105E8E0020371A90063DE0FF123E3490063EE0F5B4
:105E9E001AE4F51ED237C262C257C24A22304A599C
:105EAE00306213152EE52ED39400506BC2CAC26217
:105EBE00D257851A2E2230570E152EE52ED394006A
:105ECE005055C262C25722AF1C151CEF7007C24A52
:105EDE00C237F53D22E51D30E005851A2E8008E516
:105EEE001A75F003A4F52EAF1D7801EF088001039B
:105EFE00D8FDF51DD262D2CA22E53F25E0246DF50C
:105F0E0082E43469F583E493FA740193FBEA540F47
:075F1E00F51CEBF51DD24A52
:015F25002259
:107AC600C3EF648094A15008EF25E025E0F52E224F
:047AD600E4F52E2283
:10740700BF010790063E7418F022BF020790063EA0
:107417007412F022BF030590063E8014BF04079044
:10742700063E740BF02290063EBF05047409F02255
:04743700740CF022BF
:103E3400EF14B420004003023F87903E4C75F0031A
:103E4400A4C58325F0C58373023EAC023EB3023E93
:103E5400BA023EC1023EC8023ECF023ED6023EDD59
:103E6400023EE4023EEB023EF2023EF9023F000251
:103E74003F07023F0E023F15023F1C023F23023F51
:103E84002A023F31023F38023F3F023F46023F4D84
:103E9400023F54023F5B023F62023F69023F6B02F2
:103EA4003F72023F79023F8075CB8E75CAC6227578
:103EB400CB9575CA772275CB9B75CA692275CBA041
:103EC40075CABA2275CBA675CA332275CBAB75CA2F
:103ED400632275CBB075CA022275CBB475CAA3220E
:103EE40075CBB875CAFA2275CBBC75CAD82275CB06
:103EF400C075CAA82275CBC475CA362275CBC775DE
:103F0400CA862275CBCA75CABC2275CBCD75CAB414
:103F14002275CBD075CA762275CBD375CA3022757B
:103F2400CBD575CAB22275CBD875CA132275CBDA34
:103F340075CA522275CBDC75CA7D2275CBDD75CA74
:103F44006E2275CBE075CA542275CBE275CA1B226A
:103F540075CBE375CAC32275CBE575CA5E2275CBF2
:103F6400E675CADA22801C75CBE875CA902275CB37
:103F7400EA75CAD92275CBEC75CA092275CBED75E1
:0A3F8400CA292275CBE875CA412254
:10716800EFC39400403FEF9408503AE4FEEF75F007
:1071780008A42428F582E43400F583E5822EF582FC
:10718800E43583F583E0FCED75F008A424E8F58286
:10719800E4341AF583E5822EF582E43583F583EC31
:0571A800F00EBE08C856
:0171AD0022BF
:105FBC008F5BE55B6405701D200A0DD20A7FF47EB1
:105FCC00011279FAC20A8074C20A7FF47E01127936
:105FDC00FAD20A8067E55B6406701D200B0DD20BAC
:105FEC007FF47E011279FAC20B800BC20B7FF47E18
:105FFC00011279FAD20B8044E55B6407701D200F07
:10600C000DD20F7FF47E011279FAC20F800BC20FF2
:10601C007FF47E011279FAD20F8021E55B6408705F
:10602C0022200D0DD20D7FF47E011279FAC20D8063
:10603C000BC20D7FF47E011279FAD20D7FF47E0132
:04604C001279FA22A9
:104D7400A233B330B401B350357D017F0812628889
:104D84005027A233B35010A2B4B3500B900652E094
:104D9400FF7C077D30800F30330F30B40C90065306
:104DA400E0FF7C077D50127234A2B4B39233A23474
:104DB400B330B501B350357D027F081262885027A5
:104DC400A234B35010A2B5B3500B900654E0FF7C4C
:104DD400077D70800F30340F30B50C900655E0FF1E
:104DE4007C077D90127234A2B5B39234A235B330ED
:104DF400B701B350357D037F081262885027A2356E
:104E0400B35010A2B7B3500B900656E0FF7C077D59
:104E1400B0800F30350F30B70C900657E0FF7C0799
:104E24007DD0127234A2B7B39235A236B330B60134
:104E3400B350357D047F081262885027A236B350E0
:104E440010A2B6B3500B900658E0FF7C077DF080AB
:104E54000F30360F30B60C900659E0FF7C087D10F9
:094E6400127234A2B6B392362298
:1075F300900027E0FF30E404D20A8002C20AEF3091
:10760300E504D20B8002C20BEF30E604D20F8002F6
:0B761300C20FEF30E703D20D22C20DC2
:01761E002249
:10739C0090063CE0FF602E20370F6029123E34D25D
:1073AC00CAD237D262752E1422E52ED39400400334
:1073BC00152E22206208D2CA752E14D26222C2CA9D
:0673CC00752E7DC2622255
:1073D2002037127F1C123E34D2CAD237D262752EA7
:1073E20064751B3C22E52ED394004003152E22AF78
:1073F2001B151BD3EF648094804004752E6422C257
:0474020037E4F53D39
:017406002263
:104E6D0020371C754006E53E75F008A424E8F58250
:104E7D00E4341AF583E06003D23722E4F53D22E5F0
:104E8D002ED394004003152E22C2CA1540E54014BE
:104E9D007003024F2814606F14604014602E14606C
:104EAD0003024F5CE53E75F008A424E8F582E43476
:104EBD001AF583E0FF7003F53D22123E34E53E7591
:104ECD00F008A424E9F582E4341A8079E53E75F002
:104EDD0008A424EAF582E4341A80397408441B705E
:104EED0003F53D22E53E75F008A424EBF582E4348C
:104EFD001AF583E0FF123E34E53E75F008A424EC6C
:104F0D00F582E4341A803EE53E75F008A424EDF5F3
:104F1D0082E4341AF583E0FF027AC67420441B70D4
:104F2D0003F53D22E53E75F008A424EEF582E43448
:104F3D001AF583E0FF123E34E53E75F008A424EF28
:104F4D00F582E4341AF583E0FF127AC6D2CA22E460
:074F5D00F53DC2CAC2372274
:10743B00E53D14601C14601C14601C14601F146068
:10744B001F2405701EC2CAC237C262C257E4F54080
:10745B0022024E6D02739C125227D258220273D213
:04746B00125E8E22FD
:10759900E52365437004E5226542601F8522428523
:1075A9002343C2A4D2A5C2A6C2A700AF23127A5F01
:0D75B900E522FF127A5F00D2A7D322C32281
:1079C200E52465446014852444D2A4D2A5C2A6C28B
:0C79D200A7AF24127A5FD2A7D322C322F1
:1079DE00E521653C601485213CD2A4C2A5C2A6C295
:0C79EE00A7AF21127A5FD2A7D322C322D8
:1040D300E4F54CF54D754E1E754FFF854D82854CAD
:1040E30083E0F5506350FFE550F0E0655060031244
:1040F3007B566350FF854D82854C83E550F0E06528
:10410300506003127B56054DE54D7002054CE54F9B
:10411300154F7002154ED3E54F9400E54E940050B1
:10412300BAE4F54CF54DF54EF54FE54D254FF582C7
:10413300E54C354EF583E4F0054FE54F7002054E2F
:10414300B4FFE7E54EB41EE275985A758921758868
:1041530045758845758DE775878075C90275331B6D
:1041630075341075351B75366075371B7538B0752A
:10417300391C753A0075B701D2A9D2A8D2AA900604
:1041830000E0FFA3E0901CE0CFF0A3EFF090060265
:10419300E0FFA3E0901CE2CFF0A3EFF0900604E071
:1041A300FFA3E0901CE4CFF0A3EFF0900606E0FF3E
:1041B300A3E0901CE6CFF0A3EFF0901CFA7417F085
:1041C300A37499F0901CFC7417F0A37499F0901CDD
:1041D300FE7417F0A37499F0901D007417F0A37484
:0941E30099F0D291D2AF1276A13D
:0141EC0022B0
:027B560080FEAF
:1074D600C2AFC284D285BF060AC286E580A2E19207
:1074E600698018BF070AC286E580A2E29269800B0E
:1074F600BF0808C286E580A2E39269D286D2AFA20F
:01750600691B
:017507002261
:10628800BF0107900020E0FE8048BF020790002170
:10629800E0FE803EBF0307900022E0FE8034BF048A
:1062A80007900023E0FE802ABF0507900024E0FE47
:1062B8008020BF0607900025E0FE8016BF070790E4
:1062C8000026E0FE800CBF0807900027E0FE800251
:1062D800E4FEBD0103EE1322BD0204EEA2E122BDDD
:1062E8000304EEA2E222BD0404EEA2E322BD0504EB
:1062F800EEA2E422BD0604EEA2E522BD0704EEA24A
:07630800E622BD0802EE339E
:01630F00226B
:024F64008F4D6F
:104F66009000B0E0F54EE54D64017037E54E240241
:104F7600FFE433FE7868E66F7001EE600302505975
:104F86007410254EF582E4341BAF82F5508F51D252
:104F9600697F011259FF127988123831C2697F017F
:104FA600025056E54D64027037E54E2402FFE433A5
:104FB600FE7869E66F7001EE600302505974602551
:104FC6004EF582E4341BAF82F5508F51D2697F02D1
:104FD6001259FF127988123831C2697F020250567F
:104FE600E54D64037033E54E2402FFE433FE786A30
:104FF600E66F7001EE705C74B0254EF582E4341BEA
:10500600AF82F5508F51D2697F031259FF1279880A
:10501600123831C2697F038037E54D64047034E588
:105026004E2402FFE433FE786BE66F7001EE7023C8
:105036007400254EF582E4341CAF82F5508F51D2B0
:10504600697F041259FF127988123831C2697F04C8
:035056001259FFED
:015059002234
:043831008F4FE4FDD4
:023835008D57AD
:1038370075F020EFA42460F582E5F03403AF82F53C
:103847005A8F5BF583E0F558D3940050030239BDD6
:10385700E558941040030239BDE557704C7FF47E5C
:10386700011279FAE55825E0F558755901E558240C
:1038770001FFE433FEC3E5599FEE6480F874809836
:1038870040030239BDE55B2559F582E4355AF583D6
:10389700E0FFE55B2559F582E4355AF583A3E0FDA2
:1038A7001276770559055980C4E5576401707AC2C5
:1038B7002B7FF47E011279FAE55825E0F558755902
:1038C70001E5582401FFE433FEC3E5599FEE648008
:1038D700F874809840030239BDE55B2559F582E409
:1038E700355AF583E0FFE55B2559F582E4355AF54E
:1038F70083A3E0FD12767790001FE0FF30E00630EB
:103907004903C22022EF30E106304D03C22122EFE6
:1039170030E206305103C22222EF30E3063054036F
:10392700C22322055905598098E5576402600302AE
:1039370039BDC22BC22CC22DC22E7FF47E01127953
:10394700FAE55825E0F558755901E5582401FFE4D3
:1039570033FEC3E5599FEE6480F87480985057E5AD
:103967005B2559F582E4355AF583E0FFE55B255978
:10397700F582E4355AF583A3E0FD12767790001FB0
:10398700E030E005303902802290001FE030E10589
:10399700303A02801690001FE030E205303B02808B
:1039A7000A90001FE030E308303C05C22002736430
:0639B7000559055980943A
:0139BD0022E7
:02452A008F4DB3
:10452C00C2659000A8E0FFE54DB401167868E6FE80
:10453C00D39F400EEE9FF55074102FF582E4341B80
:10454C00804FE54DB402167869E6FED39F400EEE1F
:10455C009FF55074602FF582E4341B8034E54DB424
:10456C000316786AE6FED39F400EEE9FF55074B0AA
:10457C002FF582E4341B8019E54DB4041C786BE6EE
:10458C00FED39F4014EE9FF55074002FF582E43457
:10459C001CAF82F5518F52D26520650302463AD288
:1045AC0069AF4D1259FF7FF47E011279FA7D207F9D
:1045BC00051276777D1A7F081276777FC87E0012F7
:1045CC0079FAE4F54EE54EC39550505B0552E55231
:1045DC00AE517002055114F5828E83E0F54F6036B2
:1045EC0024F5601414601714601A14601D146020F4
:1045FC0024057028E4FD80277D5F7F0780227D5E87
:10460C007F06801C7D0A7F0280167D327F0280101F
:10461C007D467F02800A7D0A7F038004AD4FE4FF54
:0E462C00127677054E809EC269AF4D1259FF7F
:01463A00225D
:1076F40030290F900671E0FF7C0B7D10127234B2BA
:107704002922202912900670E0FF7C0A7DF0127273
:0877140034B229E4786CF6227E
:105F26007D3F7F091276777D507F08127677900045
:105F36000EE493FDE4FF1276777D5B7F061276779B
:105F460090000FE493FDE4FF127677900010E4933F
:105F5600FDE4FF127677900011E49324BFB40800A5
:105F66005053905F7675F003A4C58325F0C58373FF
:105F7600025F8E025F92025F96025F9C025FA20240
:105F86005FA8025FAE025FB47D0A80067D328002A2
:105F96007D467F02801C7D0A7F0380167D287F0355
:105FA60080107D467F03800A7D0A7F0480047D2859
:065FB6007F041276772241
:10776C008F53D2691259FF7D4B7F021276777D04BD
:10777C00E4FF1276777D387F04127677125F26C28B
:07778C0069AF531259FF22FF
:0B798800855182855083E0FFA3E0FDE5
:10799300BF0A02E4FFBD0A02E4FDEF75F00AA42D5D
:0279A300FF22C1
:10530200C265D208D2207FF47E011279FA7D2E7F07
:10531200031276777D607F02127677C208C220126E
:10532200331E7F081274D640030253CE3049F01266
:10533200331E2049FA7868E6640770427E007F7067
:1053420075331B7534108F828E837407F07D01E5EF
:10535200342DF582E43533F583E58224FFF582E5C9
:105362008334FFF583E0F9EF2DF582E43EF583E91E
:10537200F00DBD08DAD2657F647E001279FA7F08EB
:105382001274D65047206503025304D208D2207FFC
:10539200F47E011279FA7D607F021276777D327F88
:1053A200061276777D1E7F05127677C208C2207CB0
:1053B200007D707B087F787E001267707F08127410
:1053C200D650097F327E001279FA80F0126C377F54
:0653D200647E001279FA6E
:0153D80022B2
:1076CB00E4F53DC258C258F532302F05C22FC23FE8
:1076DB0022303005C230C24122303105C231C243A3
:0976EB0022303204C232C24522F1
:1041ED007580FFC286E580540FFFC285E580C454FB
:1041FD00F04FF520D2867D027F0112628840107D3E
:10420D00037F011262884007300004D23980287D77
:10421D00027F01126288500A300007300104D23942
:10422D0080157D037F01126288500A200003300142
:10423D0004D2398002C2397D027F02126288401099
:10424D007D037F021262884007300204D23A802833
:10425D007D027F02126288500A300207300304D2B9
:10426D003A80157D037F02126288500A20020330C6
:10427D000304D23A8002C23A7D027F031262884063
:10428D00107D037F031262884007300404D23B8007
:10429D00287D027F03126288500A3004073005041E
:1042AD00D23B80157D037F03126288500A200403E0
:1042BD00300504D23B8002C23B7D027F041262882E
:1042CD00400F7D037F041262884006300603D23C06
:1042DD00227D027F041262885009300606300703E2
:1042ED00D23C227D037F04126288500920060330E0
:0742FD000703D23C22C23C82
:014304002296
:10331E00202B6A20391C205019901CFAE07002A351
:10332E00E0700B7D067F011262885002D247C249BF
:10333E00804B30392130501E901CE0E07002A3E02B
:10334E00700B7D087F011262885002D23D306302FD
:10335E00D259D2498027303908205005126C378057
:10336E001C203919305016C249C250C214C210C2A4
:10337E001CC2181277BA7868E66002D259202C71F6
:10338E00203A1C205319901CFCE07002A3E0700B35
:10339E007D067F021262885002D24BC24D8052309F
:1033AE003A28305325901CE2E07002A3E070127DA3
:1033BE00087F0212628850097F021277935002D260
:1033CE003E306402D259D24D8027303A0820530540
:1033DE00126C8B801C203A19305316C24DC253C248
:1033EE0015C211C21DC2191279317869E66002D276
:1033FE005A202D71203B1C205519901CFEE07002A6
:10340E00A3E0700B7D067F031262885002D24EC27B
:10341E00518052303B28305525901CE4E07002A3B9
:10342E00E070127D087F0312628850097F031277C5
:10343E00935002D240302802D259D2518027303BCD
:10344E0008205505126CDF801C203B19305516C222
:10345E0051C255C216C212C21EC21A12794E786AD3
:10346E00E66002D25B202E6D203C1B205618901D6C
:10347E0000E07002A3E0700B7D067F04126288509C
:10348E0002D252C25422303C27305624901CE6E021
:10349E007002A3E070127D087F0412628850097FCB
:1034AE00041277935002D242302A02D259D25422B9
:1034BE00303C06205603026D33203C19305616C29E
:1034CE0054C256C217C213C21FC21B12796B786B3D
:0634DE00E66002D25E224E
:047B4F0012505A2254
:10505A0090001FE0540FFFBF010B304906203D03AB
:10506A00025121C322EF64037014304906203D0324
:10507A00025121304D06203E0302512CC322EF6417
:10508A00057014304906203D030251213051062093
:10509A004003025137C322EF6409701330490520D7
:1050AA003D028073305406204203025142C322EF6C
:1050BA006407701A304905203D02805B304D052097
:1050CA003E02805E3051052040028061C322EF64B7
:1050DA000B701A304905203D02803C304D05203EB8
:1050EA0002803F305405204202804DC322EF640DF6
:1050FA00701A304905203D02801D305105204002BA
:10510A00802B305405204202802EC322EF640F7098
:10511A002E304908203D05753E01D322304D082026
:10512A003E05753E02D322305108204005753E03E4
:10513A00D322305408204205753E04D322C322C329
:01514A002242
:10779300BF010690001FE01322BF020790001FE005
:1077A300A2E122BF030790001FE0A2E222BF04066A
:0777B30090001FE0A2E32299
:106C37007868E6602275331B753410E4FFE5342F5E
:106C4700F582E43533F583E4F00FBF50F075331B5D
:106C5700753410E47868F6900600E0FFA3E0901C16
:106C6700E0CFF0A3EFF0900608E0FFA3E0901CFA56
:106C7700CFF0A3EFF0C246C247C25DC23DC263C2B6
:036C87003FD250A9
:016C8A0022E7
:106C8B007869E6602275351B753660E4FFE5362FB3
:106C9B00F582E43535F583E4F00FBF50F075351B05
:106CAB00753660E47869F6900602E0FFA3E0901C6D
:106CBB00E2CFF0A3EFF090060AE0FFA3E0901CFCFC
:106CCB00CFF0A3EFF0C248C24BC25FC23EC264C258
:036CDB0041D25350
:016CDE002293
:106CDF00786AE6602275371B7538B0E4FFE5382F08
:106CEF00F582E43537F583E4F00FBF50F075371BAD
:106CFF007538B0E4786AF6900604E0FFA3E0901CC4
:106D0F00E4CFF0A3EFF090060CE0FFA3E0901CFEA1
:106D1F00CFF0A3EFF0C24CC24EC260C240C228C235
:036D2F0043D255F7
:016D3200223E
:106D3300786BE6602275391C753A00E4FFE53A2F5B
:106D4300F582E43539F583E4F00FBF50F075391C53
:106D5300753A00E4786BF6900606E0FFA3E0901C1A
:106D6300E6CFF0A3EFF090060EE0FFA3E0901D0046
:106D7300CFF0A3EFF0C24FC252C261C242C22AC2D5
:036D830045D256A0
:016D860022EA
:10594A00C208C209C20EC20C1279DEC265D25CE478
:10595A00F53D7FE87E031279FAC298C2AF75567F89
:10596A00755596755498755300785374FF12592CCF
:10597A00E4FBFAF9F8C3125919504430983E120060
:10598A0006127B11EF14601824F0602624C1600B04
:10599A0024F670287F06127B3F80211270D8801C63
:1059AA007F06127B3F12746F1275F3126F1BD2655A
:1059BA00800A7F06127B3F1266FFD2653065AAE431
:1059CA00786CF6D2697F011259FF7F01126B377D1D
:1059DA00467F021276777D1E7F071276777D147FC7
:1059EA00081276777D327F03127677C2697F0112B9
:0459FA0059FFC25C33
:0159FE002286
:1066FF00756701756500756620E4F5577F02127B9B
:10670F003FE5672402F559AF67127B3FE4F558E583
:10671F00662558F582E43565F583E0FF127B3FE58A
:10672F00662558F582E43565F583E02559F5590559
:10673F0058E558C3948040D7AF59127B3F7F03125F
:10674F007B3F127B47EF64156016056774802566E3
:10675F00F566E43565F5650557E557C39435409CF7
:01676F002207
:10746F00756701756500756620E4F5571275C6508E
:10747F00077F06127B3F80057F15027B3F056774F0
:10748F00802566F566E43565F5650557E557C394C0
:03749F003540D99C
:0174A20022C7
:1075C600E4F558127B4774502558F582E4341CF5CF
:1075D60083EFF00558E558C3948440E7127A759016
:0C75E6001CD2E0B50705127896D322C332
:0175F2002276
:10789600E4FF74522FF582E4341CF583E0FEE566BE
:0F78A6002FF582E43565F583EEF0000FBF80E328
:0178B50022B0
:107A7500E4FFFE74502EF582E4341CF583E02FFFFD
:047A85000EBE82EFC0
:017A890022DA
:1070D800E4F557F55D755CE0755B93755A04F559F1
:1070E800785974FF12592CE4FBFAF9F8C3125919AC
:1070F80050253098EB1200068F58E5586404601745
:10710800AF5D055D74502FF582E4341CF583E558B6
:07711800F02557F55780C96F
:01711F00224D
:04000600AF99C29854
:01000A0022D3
:087B3F003099FDC2998F9922D3
:077B47003098FDAF99C298D0
:017B4E002214
:105B670007010203040506070707060504030201E8
:105B770003010A0A03020A0A03030A0A03040A0AB8
:105B8700030307050303020503070A0A04024B0080
:105B9700040438072E03024B0004043802055F0093
:105BA7000302055F000402055F000502055F0006AA
:105BB70002055F000702055F000802055F00090292
:105BC700055F000A02055F000B02055F000C020576
:105BD7005F000D02055F000E02055F000F02055F03
:105BE700001002055F001102055F001204072E086E
:105BF700260640033204072E082606400253080CE7
:075C07000A1D040000241B2C
:10001600C2AF9000207491F09000217481F090009E
:1000260022F0900023F09000247403F090002574D1
:10003600BFF09000267408F0900027740FF090002F
:10004600307409F0A37403F0E4A3F0A37410F0A3D2
:100056007403F0E4A3F0A37415F0A37403F0A3747F
:1000660015F0A37403F0E4A3F0A37410F0A37403D3
:10007600F0E4A3F0A37409F0A37403F0A37415F0DD
:10008600A37403F0A314F0A3741AF0A37403F0E4AA
:10009600A3F0A3F0A3F0A3741AF0A37403F0A314BF
:1000A600F0A37415F0A37403F0E4A3F0A3F0A3F097
:1000B6007E5B7F777C007D807B041271F37E5B7FA5
:1000C6007B7C007D887B041271F37E5B7F7F7C00E6
:1000D6007D907B041271F37E5B7F837C007D987B31
:1000E600041271F37E5B7F8B7C007DA07B04127112
:1000F600F37E5B7F877C007DA87B041271F37E5BB9
:100106007F8F7C007DB07B041271F37E5B7F677C02
:10011600007D707B081271F37E5B7F6F7C007D78BB
:100126007B081271F37E5B7F937C037D807B0912D3
:1001360071F37E5B7F9C7C037DA07B071271F37E4F
:100146005B7FA37C037DC07B051271F37E5B7FA87A
:100156007C037DE07B051271F37E5B7FAD7C047DC5
:10016600007B051271F37E5B7FB27C047D207B05EC
:100176001271F37E5B7FB77C047D407B051271F3C1
:100186007E5B7FBC7C047D607B051271F37E5B7FAA
:10019600C17C047D807B051271F37E5B7FC67C0487
:1001A6007DA07B051271F37E5B7FCB7C047DC07BDB
:1001B600051271F37E5B7FD07C047DE07B051271B6
:1001C600F37E5B7FD57C057D007B051271F37E5B3C
:1001D6007FDA7C057D207B051271F37E5B7FDF7CF9
:1001E600057D407B051271F37E5B7FE47C057D60B7
:1001F6007B051271F37E5B7FE97C057D807B0512B2
:1002060071F37E5B7FEE7C057DA07B051271F37E2C
:100216005B7FF37C057DC07B091271F37E5B7FFCFF
:100226007C057DE07B091271F3900600E4F0A3746F
:10023600B4F0900602E4F0A374B4F0900604E4F07F
:10024600A374B4F0900606E4F0A374B4F090061814
:100256007401F0A374E0F090061AE4F0A37478F049
:1002660090061EE4F0A3743CF09006087402F0A316
:100276007458F090060A7402F0A37458F090060CB5
:100286007402F0A37458F090060E7402F0A374582A
:10029600F09006107401F0A3742CF090061274020C
:1002A600F0A37458F09006147403F0A37484F090CD
:1002B60006167404F0A374B0F07407900620F0A339
:1002C600F0900622F0A3F090061C7402F0A3745876
:1002D600F0900630740AF09006317428F0900633D8
:1002E600740AF0900634F09006327405F07E5C7F56
:1002F600057C067D407B091271F390063D7417F06C
:1003060090063E740CF090063C7419F0E490063F9B
:10031600F090063B740CF09006527401F090073092
:100326007469F0A37411F09006537401F0900750AD
:100336007469F0A37410F09006547401F09007707D
:100346007469F0A37421F09006557401F09007903B
:100356007469F0A37420F09006567401F09007B00B
:100366007469F0A37431F09006577401F09007D0C9
:100376007469F0A37430F09006587401F09007F099
:100386007469F0A37441F09006597401F090081056
:100396007469F0A37440F090065A7401F090083026
:1003A6007462F0A37411F0A37432F0A37401F0A385
:1003B6007450F0A37410F090065B7401F09008502E
:1003C6007461F0A37420F0A37462F0A37411F0A317
:1003D6007432F0A37402F0A37450F0A37410F0907A
:1003E600065C7401F09008707451F0A37411F0A3C8
:1003F6007433F0A3E4F0A37451F0A37410F09006E4
:100406005D7401F09008907462F0A37411F0A37407
:1004160030F0A37402F0A37462F0A37410F0900697
:100426005E7401F09008B07451F0A37411F0A374D7
:1004360041F0A37410F0A37451F0A37410F0900669
:100446005F7401F09008D07451F0A37411F0A37496
:1004560034F0A37414F0A37451F0A37410F0900652
:10046600607401F09008F07451F0A37411F0A37455
:1004760034F0A37418F0A37451F0A37410F090062E
:10048600617401F09009107451F0A37411F0A37413
:1004960034F0A37428F0A37451F0A37410F09006FE
:1004A600627401F09009307462F0A37411F0A374C1
:1004B60030F0A37403F0A37462F0A37410F09006F6
:1004C600637401F09009507462F0A37411F0A37480
:1004D60030F0A37404F0A37462F0A37410F09006D5
:1004E600647401F09009707462F0A37411F0A3743F
:1004F60060F0A37401F0A37495F0A3743DF0A374A7
:1005060090F0A37401F0A37498F0A37426F0A3747A
:1005160096F0A37440F0A37462F0A37410F0A37471
:1005260061F0A37470F09006657401F09009907400
:1005360062F0A37411F0A37460F0A37401F0A374C5
:1005460095F0A3743DF0A37490F0A37401F0A37426
:1005560096F0A37438F0A37462F0A37410F09006BA
:10056600667401F09009B07462F0A37411F0A3747C
:1005760060F0A37401F0A37495F0A3743DF0A37426
:1005860090F0A37402F0A37498F0A37426F0A374F9
:1005960096F0A37440F0A37462F0A37410F0A374F1
:1005A60061F0A37470F09006677401F09009D0743E
:1005B60062F0A37411F0A37460F0A37401F0A37445
:1005C60095F0A3743DF0A37490F0A37402F0A374A5
:1005D60096F0A37438F0A37462F0A37410F090063A
:1005E600687401F09009F07462F0A37411F0A374BA
:1005F60060F0A37401F0A37495F0A3743DF0A374A6
:1006060090F0A37403F0A37498F0A37426F0A37477
:1006160096F0A37440F0A37462F0A37410F0A37470
:1006260061F0A37470F09006697401F0900A10747A
:1006360062F0A37411F0A37460F0A37401F0A374C4
:1006460095F0A3743DF0A37490F0A37403F0A37423
:1006560096F0A37438F0A37462F0A37410F09006B9
:100666006A7401F0900A307462F0A37411F0A374F6
:1006760060F0A37401F0A37495F0A3743DF0A37425
:1006860090F0A37404F0A37498F0A37426F0A374F6
:1006960096F0A37440F0A37462F0A37410F0A374F0
:1006A60061F0A37470F090066B7401F0900A5074B8
:1006B60062F0A37411F0A37460F0A37401F0A37444
:1006C60095F0A3743DF0A37490F0A37404F0A374A2
:1006D60096F0A37438F0A37462F0A37410F0900639
:1006E6006C7401F0900A707462F0A37411F0A37434
:1006F60060F0A37401F0A37430F0A37405F0A37442
:1007060062F0A37410F090066D7401F0900A907474
:1007160062F0A37421F0A37460F0A37401F0A374D3
:1007260030F0A37406F0A37462F0A37420F0900670
:100736006E7401F0900AB07462F0A37431F0A37481
:1007460060F0A37401F0A37430F0A37407F0A374EF
:1007560062F0A37430F090066F7401F0900AD074C2
:1007660062F0A37441F0A37460F0A37401F0A37463
:1007760030F0A37408F0A37462F0A37440F09006FE
:10078600707401F0900AF07464F0A37411F0A3740D
:1007960096F0A37432F0A37495F0A3741EF0A374BC
:1007A60098F0A3744BF0A37464F0A37410F0900651
:1007B600717401F0900B107464F0A37411F0A374BB
:1007C60096F0A37432F0A37495F0A3741EF0A3748C
:1007D60093F0A37418F0A37464F0A37410F0900659
:1007E600737401F0900B507462F0A37411F0A3744B
:1007F60060F0A37401F0A37495F0A3743DF0A374A4
:1008060090F0A37402F0A37497F0A37426F0A37477
:1008160093F0A37418F0A37462F0A37410F0A37499
:1008260070F0A37410F09006747401F0900B70745D
:1008360062F0A37411F0A37460F0A37401F0A374C2
:1008460095F0A3743DF0A37490F0A37403F0A37421
:1008560097F0A37426F0A37493F0A37418F0A3740E
:1008660062F0A37410F0A37470F0A37420F09006E5
:10087600757401F0900B907462F0A37411F0A37478
:1008860060F0A37401F0A37495F0A3743DF0A37413
:1008960090F0A37404F0A37497F0A37426F0A374E5
:1008A60093F0A37418F0A37462F0A37410F0A37409
:1008B60070F0A37430F09006817401F0900D1074FE
:1008C60062F0A37411F0A37460F0A37401F0A37432
:1008D60092F0A3744BF0A37490F0A37404F0A37485
:1008E60094F0A37438F07499A3F0A3F0A37460F0A5
:1008F600A37401F0A37462F0A37410F01222F8122C
:100906006F1BD2697F011259FF7D2F7F0712767701
:100916007D0C7F031276777D327F061276777D1EF9
:100926007F0512767790001F7401F0FD7F1F7E0011
:0B093600127274C2697F011259FF2287
:1022F8009001007402F0A3740DF0A37402F090062C
:10230800A014F09010F07464F0A37411F0A3749703
:10231800F0A3742EF0A37495F0A3743DF0A3749009
:10232800F0A37402F0A37496F0A37438F0A3746455
:10233800F0A37410F0A37470F0A37411F090010866
:102348007402F0A3740EF0A37402F09006A114F0C6
:102358009011107464F0A37411F0A37497F0A3742F
:102368002EF0A37495F0A3743DF0A37490F0A374B9
:1023780002F0A37496F0A37436F0A37464F0A37407
:1023880010F0A37470F0A37410F09001107402F0B0
:10239800A3740DF0A37403F09006A27401F09011D9
:1023A800307464F0A37411F0A37497F0A3742EF042
:1023B800A37495F0A3743DF0A37490F0A37403F094
:1023C800A37496F0A37438F0A37464F0A37410F0A7
:1023D800A37470F0A37421F09001187402F0A37430
:1023E8000EF0A37403F09006A37401F090115074DA
:1023F80064F0A37411F0A37497F0A3742EF0A3747F
:1024080095F0A3743DF0A37490F0A37403F0A37443
:1024180096F0A37436F0A37464F0A37410F0A37458
:1024280070F0A37420F09001207402F0A3740DF0F2
:10243800A37404F09006A47401F09011707464F011
:10244800A37411F0A37497F0A3742EF0A37495F0FD
:10245800A3743DF0A37490F0A37404F0A37496F0F1
:10246800A37438F0A37464F0A37410F0A37470F02C
:10247800A37431F09001287402F0A3740EF0A374D1
:1024880004F09006A57401F09011907464F0A374A0
:1024980011F0A37497F0A3742EF0A37495F0A374AD
:1024A8003DF0A37490F0A37404F0A37496F0A374A1
:1024B80036F0A37464F0A37410F0A37470F0A374DE
:1024C80030F09001307403F0A3740DF0A37402F09F
:1024D800A304F09006A67401F09011B07464F0A300
:1024E8007411F0A37497F0A3742EF0A37495F0A35D
:1024F800743DF0A37490F0A37402F0A37490F0A359
:102508007403F0A37496F0A37438F0A37464F0A372
:102518007410F0A37470F0A37441F0900138740340
:10252800F0A3740EF0A37402F0A304F09006A7744D
:1025380001F09011D07464F0A37411F0A37497F0B3
:10254800A3742EF0A37495F0A3743DF0A37490F0D7
:10255800A37402F0A37490F0A37403F0A37496F02C
:10256800A37436F0A37464F0A37410F0A37470F02D
:10257800A37440F09001407404F0A3740DF0A374A8
:1025880002F0A304F0A304F09006A87401F09011DF
:10259800F07464F0A37411F0A37497F0A3742EF090
:1025A800A37495F0A3743DF0A37490F0A37402F0A3
:1025B800A37490F0A37403F0A37490F0A37404F0D0
:1025C800A37496F0A37438F0A37464F0A37410F0A5
:1025D800A37470F0A37441F0A37470F0A37451F065
:1025E8009001487404F0A3740EF0A37402F0A304DD
:1025F800F0A304F09006A97401F09012107464F02E
:10260800A37411F0A37497F0A3742EF0A37495F03B
:10261800A3743DF0A37490F0A37402F0A37490F037
:10262800A37403F0A37490F0A37404F0A37496F059
:10263800A37436F0A37464F0A37410F0A37470F05C
:0D264800A37440F0A37470F0A37450F0224E
:0A71F3008E4C8F4D8C4E8D4F8B504B
:1071FD00E4F9C3E5506480F8E96480985028E9FF0C
:10720D003395E0FEE54D2FF582E54C3EF583E49395
:10721D00FFE9FD3395E0FCE54F2DF582E54E3CF59C
:06722D0083EFF00980CCA4
:017233002238
:107A2F00D291C2A4C2A5C2A6C2A7007F05127A5FD7
:097A3F0000127A4900D2A7D2918D
:017A4800221B
:1078F500127A2FEF20E0F9D291C2A4C2A5C2A6C286
:0E790500A7007F06127A5F0000D2A7D291225F
:10791300127A2FEF20E0F9D291C2A4C2A5C2A6C267
:0E792300A7007F04127A5F0000D2A7D2912243
:046D87008E528F5346
:106D8B00AE04AF058E568F57D291C2A4C2A5C2A630
:106D9B00C2A7007F03127A5FE552FF127A5FAF53EF
:106DAB00127A5FE4F554F555127A49E5572555F5F6
:106DBB0082E5563554F583EFF00555E55570020520
:0E6DCB0054C39420E554940040DED2A7D29128
:016DD9002297
:0868AE008E5D8F5E8C5F8D6032
:1068B600127A2FEF20E0F91278F5855D63855E6424
:1068C600D291C2A4C2A5C2A6C2A7007F02127A5F55
:1068D600E55FFF127A5FAF60127A5FE4F561F562F9
:1068E600E5642562F582E5633561F583E0FF127A9A
:1068F6005F0562E56270020561C39420E56194005C
:0769060040DE00D2A7D29190
:01690D002267
:0A6770008E4C8F4D8C4E8D4F8B50D8
:10677A00C2AF1278F5127A2FEF20E0F9854E5285D2
:10678A004F53D291C2A4C2A5C2A6C2A7007F0212C9
:10679A007A5FE54CFF127A5FAF4D127A5FE4F551EA
:1067AA00AF50EF3395E0FEC3E5519FEE6480F87475
:1067BA0080985014E5532551F582E43552F583E06B
:1067CA00FF127A5F055180D800D2A7D291127913AD
:0267DA00D2AF3C
:0167DC00229A
:107274008E5B8F5C8D5DC2AF1278F5127A2FEF2092
:10728400E0F9D291C2A4C2A5C2A6C2A7007F02128D
:107294007A5FE55BFF127A5FAF5C127A5FAF5D12D3
:0E72A4007A5F0000D2A7D291127913D2AF22E6
:0477E0008E4C8F4DEF
:1077E400D291C2A4C2A5C2A6C2A77F03127A5FE542
:1077F4004CFF127A5FAF4D127A5F127A49D2A7D248
:0178040091F2
:017805002260
:10712000C2AF754E00754F20755000755120E4F5C3
:107130004CF54DAD4FAC4EAF51AE50126D87742033
:10714000254FF54FE4354EF54E74202551F551E4A9
:107150003550F550054DE54D7002054CC394D6E50C
:077160004C940040CED2AFB9
:017167002205
:106F1B00C2AF755B00755C20755900755A20E4F59E
:106F2B0057F558AD5AAC59AF5CAE5B1268AE7420D6
:106F3B00255AF55AE43559F5597420255CF55CE46E
:106F4B00355BF55B0558E55870020557C394D6E5DC
:0A6F5B0057940040CE127913D2AF14
:016F65002209
:046E2C008C4D8D4EAE
:106E3000EF6048D22BD22CD22DD22EE4F54F854EC6
:106E400082854D83E0FEA3E04E6028AF4FEF33957F
:106E5000E0FEEF25E0FFEE33FEE54E2FF582E54D37
:106E60001254AE926520650B054FC3E54F648094C4
:0B6E70009040CBC22BC22CC22DC22EC2
:016E7B0022F4
:047234008C4D8D4EA2
:10723800EF6038E4F54F854E82854D83E0FEA3E08C
:107248004E6028AF4FEF3395E0FEEF25E0FFEE33B9
:10725800FEE54E2FF582E54D1254AE926520650B82
:0B726800054FC3E54F6480949040CBBD
:0172730022F8
:0854AE003EF583E0FEA3E0FFE0
:0454B600AD07AC068C
:1054BA00C266780CEF088006A2E0CE13CE13D8F8A5
:1054CA00540FF5507808AF05AE04EF088006A2E045
:1054DA00CE13CE13D8F8540FF5517804AF05AE04A5
:1054EA00EF088006A2E0CE13CE13D8F8540FF55277
:1054FA00ED540FF553E550607CB4010BAB53AD523C
:10550A00AF511257D4806EE550B4030BAB53AD5272
:10551A00AF51126A29805EE550B4040BAB53AD5209
:10552A00AF51126F66804EE550B4050BAB53AD52C6
:10553A00AF51123CC0803EE550B4060BAB53AD529E
:10554A00AF5112180F802EE550B4070BAB53AD5272
:10555A00AF511253D9801EE550B4080BAB53AD526C
:10556A00AF51126DDA800EE550B40909AB53AD5252
:07557A00AF5112782BA2666D
:015581002207
:1057D4008F548D558B56E554B40113900020E0FF8F
:1057E4001269D1900020EFF0FD7F2002586FE5543C
:1057F400B402119000211269CB900021EFF0FD7FDB
:105804002102586FE554B403109000221269CB9022
:105814000022EFF0FD7F228052E554B40410900082
:10582400231269CB900023EFF0FD7F23803DE554E4
:10583400B405109000241269CB900024EFF0FD7F92
:10584400248028E554B406109000251269CB9000FA
:1058540025EFF0FD7F258013E554B407139000264F
:105864001269CB900026EFF0FD7F267E0002727451
:10587400E554B408169000271269CB900027EFF086
:0C588400FD7F277E001272741275F32263
:0669CB00E0FFAB56AD55E4
:1069D100D267AC07BD01047E018033BD02047E0293
:1069E100802CBD03047E048025BD04047E08801E26
:1069F100BD05047E108017BD06047E208010BD07F2
:106A0100047E408009BD08047E808002C267BB010C
:106A110005EE4204800BEB7006EEF452048002C2D4
:076A210067306703AF042298
:016A2800224B
:106A29008F548D558B56E554700BAD56AF55127A70
:106A3900F1E4FD801EE554B4010BAD56AF55127A51
:106A4900F17D01800EE554B4020CAD56AF55127AB2
:106A5900F17D02023835E554B4030AE55570061292
:106A69007364C25822E554B40410AD56AF5512668A
:0B6A7900CD8F3F753D05E53D70FC2210
:106F66008F548D558B56E5547027E555B401047D35
:106F7600018019E555B402047D028010E555B4037D
:106F8600047D038007E555B404207D04AF560271E5
:106F960068E554B40114E555D39400400DE55594C5
:0B6FA600055007753D01E53D70FC2221
:103CC0008B54EF7017BD0114E5547002C220E55407
:103CD00064016003023E2CD220023E2CEF7017BD1F
:103CE0000214E5547002C221E55464016003023EEF
:103CF0002CD221023E2CEF7017BD0314E554700244
:103D0000C222E55464016003023E2CD222023E2C02
:103D1000EF7017BD0414E5547002C223E55464012A
:103D20006003023E2CD223023E2CEF701BBD05180F
:103D3000E5547004C220C221E55464016003023ED0
:103D40002CD220D221023E2CEF701BBD0618E55468
:103D50007004C222C223E55464016003023E2CD2E7
:103D600022D223023E2CBF0117BD0114E55470027C
:103D7000C224E55464016003023E2CD224023E2C8E
:103D8000BF0117BD0214E5547002C225E554640159
:103D90006003023E2CD225023E2CBF0116BD031348
:103DA000E5547002C226E55464016003023E2CD241
:103DB000268079BF0113BD0410E5547002C227E5C7
:103DC0005464017067D2278063BF0117BD0514E5F5
:103DD000547004C224C225E5546401704FD224D229
:103DE000258049BF0117BD0614E5547004C226C2E0
:103DF00027E55464017035D226D227802FEF640165
:103E0000702AED64097025E554B401047F0180191E
:103E1000E554B402047F028010E554B403047F0328
:103E20008007E554B404057F04126B377F327E00AF
:043E30001279FA22E7
:10180F008F548D558B56E5547016AD56AF55127AD1
:10181F00F1901D14EFF0901D14E0D3940050F722B7
:10182F00E554B40117E555B40112E5567002C2082C
:10183F00E55664016003021BB5D20822E554B401DA
:10184F0017E555B40212E5567002C209E556640158
:10185F006003021BB5D20922E554B40117E555B454
:10186F000312E5567002C20EE55664016003021BB7
:10187F00B5D20E22E554B40117E555B40412E5565E
:10188F007002C20CE55664016003021BB5D20C2234
:10189F00E554B4011BE555B40516E5567004C208AE
:1018AF00C209E55664016003021BB5D208D20922B2
:1018BF00E554B40118E555B40613E5567004C20E8D
:1018CF00C20CE55664016003021BB58024E5546425
:1018DF00017023E555B4071EE5567008C208C2090A
:1018EF00C20EC20CE55664016003021BB5D208D2CA
:1018FF0009D20ED20C22E554B4021DE555B40118DD
:10190F00E5567004C208C220E55664016003021B4D
:10191F00B5D208D220021AD5E554B4021DE555B44C
:10192F000218E5567004C209C221E556640160032E
:10193F00021BB5D209D221021A61E554B4021DE58A
:10194F0055B40318E5567004C20EC222E556640161
:10195F006003021BB5D20ED222021A85E554B402DF
:10196F001DE555B40418E5567004C20CC223E556A4
:10197F0064016003021BB5D20CD223021AA8E554EE
:10198F0064027026E55564057020E5567008C2089C
:10199F00C209C220C221E55664016003021BB5D201
:1019AF0008D209D220D221021AD5E554640270263A
:1019BF00E55564067020E5567008C20EC20CC222AF
:1019CF00C223E55664016003021BB5D20ED20CD2BE
:1019DF0022D223021A85E55464027035E555640757
:1019EF00702FE5567010C208C209C20EC20CC22079
:1019FF00C221C222C223E55664016003021BB5D285
:101A0F0008D209D20ED20CD220D221D222D22380D8
:101A1F0065E554B4031DE555B40118E5567004C2CD
:101A2F0008C224E55664016003021BB5D208D22414
:101A3F00021AD5E554B4031FE555B4021AE55670E2
:101A4F0004C209C225E55664016003021BB5D20921
:101A5F00D2257F02021B04E554B4031EE555B403DF
:101A6F0019E5567004C20EC226E5566401600302E2
:101A7F001BB5D20ED2267F03807BE554B4031EE53F
:101A8F0055B40419E5567004C20CC227E55664011B
:101A9F006003021BB5D20CD2277F048058E5546433
:101AAF00037027E55564057021E5567008C208C21A
:101ABF0009C224C225E55664016003021BB5D20892
:101ACF00D209D224D2257F01802BE55464037028DC
:101ADF00E55564067022E5567008C20EC20CC22688
:101AEF00C227E55664016003021BB5D20ED20CD299
:101AFF0026D2277F03026B37E554B4040AE555B4A9
:101B0F000105AF56026593E554B4040AE555B402D6
:101B1F0005AF56026846E5546409701EE555B401D9
:101B2F0019E5567003C20A22E556B40103D20A2200
:101B3F00E556640270707F058069E5546409701E74
:101B4F00E555B40219E5567003C20B22E556B401F0
:101B5F0003D20B22E5566402704C7F068045E55494
:101B6F006409701EE555B40319E5567003C20F22C0
:101B7F00E556B40103D20F22E556640270287F07A1
:101B8F008021E5546409701EE555B40419E55670BB
:101B9F0003C20D22E556B40103D20D22E556B4025D
:071BAF00057F08125FBC2254
:1053D900AC07EC600302548FBD010CEB700990001F
:1053E9001FE054FDF0800DBD010ABB010790001FAD
:1053F900E04403F0BD020CEB700990001FE054FB80
:10540900F0800DBD020ABB010790001FE04405F0C2
:10541900BD030CEB700990001FE054F7F0800DBD3F
:10542900030ABB010790001FE04409F0BD040CEB1F
:10543900700990001FE054F9F0800DBD040ABB010A
:105449000790001FE04407F0BD050CEB70099000C0
:105459001FE054F3F0800DBD050ABB010790001F42
:10546900E0440DF0BD060CEB700990001FE054F10B
:10547900F08025ED64067020EB6401701B90001F1D
:10548900E0440FF08012BC010FED700CEB7004C208
:10549900298005BB0102D22990001FE0FD7F1F7EF4
:0554A9000012727422E4
:106DDA008F548D558B56E554700C127AED744F2FE3
:106DEA00F58274068020E554B4010C127AED744FD2
:106DFA002FF58274068024E554B40210127AED74D9
:106E0A009F2FF58274063EF583E4F022E554B4031D
:106E1A0010127AED749F2FF58274063EF583740181
:026E2A00F02254
:02782B008F5478
:10782D00AF057804EF08800123D8FD4BF555E554DD
:10783D00B40908E555B49903025F26AD55AF54124E
:02784D0076774C
:01784F002216
:10659300E545B40109BF0106D220D2088060E54574
:1065A300B40109EF7006C220C2088052E545B40267
:1065B30009BF0106D221D2098044E545B40209EF9F
:1065C3007006C221C2098036E545B40309BF01063E
:1065D300D222D20E8028E545B40309EF7006C22209
:1065E300C20E801AE545B40409BF0106D223D20CBA
:1065F300800CE545B40407EF7004C223C20C127982
:0A660300DEAF3E126B371279C2229F
:10684600E545B40108BF0105D224D20822E545B4C6
:106856000108EF7005C224C20822E545B40208BF4C
:106866000105D225D20922E545B40208EF7005C21A
:1068760025C20922E545B40308BF0105D226D20E7A
:1068860022E545B40308EF7005C226C20E22E5458F
:10689600B40408BF0105D227D20C22E545B404078B
:0868A600EF7004C227C20C22AE
:047AED00AD56AF558E
:0D7AF100EF75F00AA47C002DFFEC35F0FECF
:017AFE002265
:020941008F4DD8
:10094300C266E4F53DD25CD2691259FF7D4B7F024A
:100953001276777D04E4FF1276777D387F04127672
:10096300777D607F0212767790061CE0FFA3E0900C
:100973001CE8CFF0A3EFF0C269AF4D1259FFE4F5C5
:1009830046C20812331EE54DB40106A249926580A2
:100993001FE54DB40206A24D92658014E54DB403E4
:1009A30006A25192658009E54DB40404A2549265F0
:1009B300901CE8E07002A3E07005D266020F8B3052
:1009C30065C112331EE54DB40106A2499265801F2D
:1009D300E54DB40206A24D92658014E54DB40306BD
:1009E300A25192658009E54DB40404A25492652096
:1009F30065D0E54DB4010A754E1B754F10786880BC
:100A03002BE54DB4020A754E1B754F607869801C47
:100A1300E54DB4030A754E1B754FB0786A800DE53A
:100A23004DB4040B754E1C754F00786BE6F550E51D
:100A330050D394005003020F85854F82854E83E087
:100A4300640B6003020F80A3E0FFB40A0AE550B40D
:100A53000205D266020F85EF64017032854F8285ED
:100A63004E83A3A3E064037025E550B40520854FAE
:100A730082854E83A3A3A3E0FFE54F2404F582E41C
:100A8300354EF583E0FDAB4D123F8E020F85854F4A
:100A930082854E83A3E0B40121854F82854E83A3D3
:100AA300A3E0B40415E550D39405400EAB4DAD4F10
:100AB300AC4EAF501234E4020F85854F82854E83CE
:100AC300A3E064017032854F82854E83A3A3E06463
:100AD300057025E550B40520854F82854E83A3A379
:100AE300A3E0FFE54F2404F582E4354EF583E0FDF2
:100AF300AB4D126513020F85854F82854E83A3E0AC
:100B030064017032854F82854E83A3A3E06406702F
:100B130025E550B40520854F82854E83A3A3A3E02A
:100B2300FFE54F2404F582E4354EF583E0FDAB4D3C
:100B3300125C0E020F85854F82854E83A3E0B401BC
:100B430021854F82854E83A3A3E0B40715E550D3D7
:100B53009405400EAB4DAD4FAC4EAF50124C7802E6
:100B63000F85854F82854E83A3E064017032854FE4
:100B730082854E83A3A3E064087025E550B4052065
:100B8300854F82854E83A3A3A3E0FFE54F2404F59D
:100B930082E4354EF583E0FDAB4D126A84020F8586
:100BA300854F82854E83A3E0B40219854F82854E1B
:100BB30083A3A3E0B4080DE550B40308AF4D127648
:100BC3004B020F85854F82854E83A3E06402702418
:100BD300854F82854E83A3A3E0B40818E550B4047F
:100BE30013854F82854E83A3A3A3E0FFAD4D1277F8
:100BF30044020F85854F82854E83A3E0B402198595
:100C03004F82854E83A3A3E0B4090DE550B40308D6
:100C1300AF4D12761F020F85854F82854E83A3E069
:100C230064027024854F82854E83A3A3E0B4091820
:100C3300E550B40413854F82854E83A3A3A3E0FF3D
:100C4300AD4D12771C020F85854F82854E83A3E03D
:100C530064037036854F82854E83A3A3E0640A70D4
:100C630029E55064057023854F82854E83A3A3A392
:100C7300E0FFE54F2404F582E4354EF583E0FD12F1
:100C83007993AD4D125715020F85854F82854E839B
:100C9300A3E06403703E854F82854E83A3A3E06483
:100CA300017031E550D39405402A854F82854E83E8
:100CB300A3A3A3E0FFE54F2404F582E4354EF583B7
:100CC300E0FD127993854D55AB50AD4FAC4E1246B6
:100CD3003B020F85854F82854E83A3E06403703604
:100CE300854F82854E83A3A3E064027029E5506497
:100CF300057023854F82854E83A3A3A3E0FFE54FB1
:100D03002404F582E4354EF583E0FD127993AD4D6D
:100D1300127046020F85854F82854E83A3E0B4038C
:100D230019854F82854E83A3A3E0B4030DE550B428
:100D33000308AF4D1272B2020F85854F82854E8331
:100D4300A3E0B40321854F82854E83A3A3E0B404BB
:100D530015E550D39403400EAB4DAD50AF4FAE4E9F
:100D6300125DF5020F85854F82854E83A3E0B403A0
:100D730019854F82854E83A3A3E0B4050DE550B4D6
:100D83000308AF4D127AFF020F85854F82854E838C
:100D9300A3E0B4031D854F82854E83A3A3E0B4066D
:100DA30011E550B4050CAD4DAF4FAE4E12732B028F
:100DB3000F85854F82854E83A3E064037024854F9E
:100DC30082854E83A3A3E0B40718E550B4041385CA
:100DD3004F82854E83A3A3A3E0FFAD4D1278B602E5
:100DE3000F85854F82854E83A3E0B4031D854F8213
:100DF300854E83A3A3E0B40811E550B4050CAD4DB3
:100E0300AF4FAE4E127539020F85854F82854E83E3
:100E1300A3E064057022E550B4041D854F82854E1E
:100E230083A3A3E0FF854F82854E83A3A3A3E0FDA5
:100E3300AB4D122D58020F85854F82854E83A3E05B
:100E4300B40524E54F2404F582E4354EF583E0B47C
:100E53000B15E550D39405400EAB4DAD50AF4FAEDF
:100E63004E12474B020F85854F82854E83A3E06464
:100E7300067022E550B4041D854F82854E83A3A3DB
:100E8300E0FF854F82854E83A3A3A3E0FDAB4D1204
:100E93002655020F85854F82854E83A3E0B4062431
:100EA300E54F2404F582E4354EF583E0B40B15E5F4
:100EB30050D39405400EAB4DAD50AF4FAE4E1231F3
:100EC30036020F85854F82854E83A3E06409702225
:100ED300854F82854E83A3A3E0B40A16E550B4047C
:100EE30011854F82854E83A3A3A3E0FF126FB10246
:100EF3000F85854F82854E83A3E064097023854F58
:100F030082854E83A3A3E0B40117E550B404128590
:100F13004F82854E83A3A3A3E0FFAD4D12565280AB
:100F230061854F82854E83A3E0B40920854F828576
:100F33004E83A3A3E0B40214E550D39404400DAB55
:100F430050AD4DAF4FAE4E1214648036854F82853F
:100F53004E83A3E064097025854F82854E83A3A346
:100F6300E0B40317E550B40412854F82854E83A382
:100F7300A3A3E0FFAD4D126E7C80078000AF4D123E
:100F830079A5206603020986C258D269AF4D12596A
:100F9300FF7D607F021276777D327F03127677C200
:0F0FA30069AF4D1259FF126F1BE4786CF6C25CF8
:010FB200221C
:0834E4008F518C528D538B5463
:1034EC00855382855283A3A3A3E0FF8D828C83E551
:1034FC008224041266C48F55E555D3940050030200
:10350C003685E55594294003023685E551640670ED
:10351C004FD269AF541259FF7D527F05127677AFA7
:10352C0055124B76E5532405F582E43552F583E0CC
:10353C00B40112749F2555F582E43406F5837401A9
:10354C00F07D38800F749F2555F582E43406F583A1
:10355C00E4F07D367F06127677C269AF540259FFCC
:10356C00E5532406F582E43552F583E0640B6003E1
:10357C00023685E5532405F582E43552F583E0B433
:10358C000110749F2555F582E43406F5837401F01F
:10359C00800D749F2555F582E43406F583E4F0E440
:1035AC00FFFEE5532407F582E43552F583E5822EC0
:1035BC00F582E43583F583E0B40B04AF0680040E8A
:1035CC00BE08DFEF7003023685C394084003023651
:1035DC008575F008E555A424F8F582E5F03400F57E
:1035EC0083EFF07E01EF2401FDE433FCEEC39DEC90
:1035FC006480F87480985036E5532406F582E435DF
:10360C0052F583E5822EF582E43583F583E0FD7572
:10361C00F008E555A424F8F582E5F03400F583E5CF
:10362C00822EF582E43583F583EDF00E80B7E553F9
:10363C002408F582E43552F583E5822FF582E435D2
:10364C0083F583E0640B602DEF2408FEC3E5519EE7
:10365C00F55175F004125890AEF0EE701CE5532441
:10366C0007FDE43552FC7E00ED2FFBEE3CFAAD5528
:10367C007F011239BED2688002C268AF54127B310E
:01368C00221B
:107874008E5CF55DAF5BEF3395E0FEE5592FF58245
:08788400E5583EF583A3E0FF87
:0A788C00EFD3940940037F0022228D
:0839BE008F568D578A588B5972
:1039C600755B01E4F55AAF5BEF3395E0FEE5592FE1
:1039D600F582E5583EF583E0FF6409706512788C40
:1039E600755C008F5DAE5C7804EF08800633CE33DD
:1039F600CE92E0D8F8127874EF425DAE5CAF5D7897
:103A060008EF08800633CE33CE92E0D8F88E5CF508
:103A16005DAF5BEF3395E0FEE5592FF582E5583E45
:103A2600F583A3A3E0FFE55BFD3395E0FCE5592DA7
:103A3600F582E5583CF583A3A3A3E0FD1279930232
:103A46003AD9AF5BEF3395E0FEE5592FF582E5589D
:103A56003EF583E0FF12788C755C008F5DAE5C7876
:103A660004EF08800633CE33CE92E0D8F81278748D
:103A7600EF425DAE5CAF5D7804EF08800633CE336F
:103A8600CE92E0D8F88E5CF55DAF5BEF3395E0FE45
:103A9600E5592FF582E5583EF583A3A3E0FF12789A
:103AA6008CEF425DAE5CAF5D7804EF08800633CEE6
:103AB60033CE92E0D8F88E5CF55DAF5BEF3395E0E0
:103AC600FEE5592FF582E5583EF583A3A3A3E0FF53
:103AD60012788CEF425DE556701EAF5AEF3395E0D3
:103AE600FEEF25E0FFEE33FE75F020E557A424D067
:103AF600F582E5F034068021E556B4012FAF5AEF82
:103B06003395E0FEEF25E0FFEE33FE75F020E55736
:103B1600A424D0F582E5F03410F583E5822FF582F2
:103B2600E5833EF583E55CF0A3E55DF07404255B73
:103B3600F55B055AC3E55A6480949050030239CC6C
:013B4600225C
:084C78008F518C528D538B54B7
:104C8000855382855283A3A3A3E0FF8D828C83E5A5
:104C90008224041266C48F55E555D3940050030254
:104CA0004D65E55594334003024D65E5516406704A
:104CB0004FD269AF541259FF7D527F05127677AFFC
:104CC00055124B76E5532405F582E43552F583E021
:104CD000B40112744F2555F582E43406F58374014E
:104CE000F07D38800F744F2555F582E43406F58346
:104CF000E4F07D367F06127677C269AF540259FF21
:104D0000E5532406F582E43552F583E0640B7055D3
:104D1000E5532405F582E43552F583E0B4011074BF
:104D20004F2555F582E43406F5837401F0800D7447
:104D30004F2555F582E43406F583E4F074F92551E6
:104D4000F55175F004125890AFF0EF7014E553244C
:104D500006FBE43552FAAD55E4FF1239BED2688045
:104D60000DC2688009C269AF541259FFC268AF54BE
:034D7000127B3182
:014D7300221D
:023F8E008B5155
:103F90001266CD8F54E554D3940050030240CBE514
:103FA00054943340030240CBD269AF511259FF7D84
:103FB000527F05127677AF54124B76749F2554F5D5
:103FC00082E43406F583E060047D3880027D367F2C
:103FD000061276777F2C7E011279FA75F008E55487
:103FE000A424F8F582E5F03400F583E0F55270077B
:103FF0007D1B7F061276777D577F02127677E5521A
:10400000607A755301AF52EF3395E0FEEF2401FF64
:10401000E43EFEAD53ED3395E0FCC3ED9FEE6480CE
:10402000F8EC6480985055AF53EF3395E0FE75F08F
:1040300008E554A424F8F582E5F03400F583E58220
:104040002FF582E5833EF583E0B40A04E4FD802485
:10405000AF53EF3395E0FE75F008E554A424F8F56E
:1040600082E5F03400F583E5822FF582E5833EF5A5
:1040700083E0FDE4FF127677055380897F2C7E0173
:104080001279FA75F020E554A424D0F582E5F034D5
:1040900010F583E0FEA3E0FF900000EEF0A3EFF048
:1040A0004E70077D1B7F061276777D0C7F0312769C
:1040B00077900000E07002A3E06009E55414FD7FF2
:1040C00001122F4CC269AF510259FFC268AF5112A1
:0240D0007B3142
:0140D20022CB
:042F4C008F558D56BA
:102F5000E4F557E5556003022FF7AF57EF3395E0DF
:102F6000FEEF25E0FDEE33FCAF56EF3395E0FEEFCC
:102F70007805C333CE33CED8F924F0F58274063EFB
:102F8000F583E5822DF582E5833CF583E0FAA3E045
:102F9000FB780CFFAE02088006A2E0CE13CE13D859
:102FA000F8540FF5587808AF03AE02EF088006A278
:102FB000E0CE13CE13D8F8540FF559AF56EF339532
:102FC000E0FEEF7805C333CE33CED8F924F0F58296
:102FD00074063EF583E5822DF582E5833CF583E0BA
:102FE000FCA3E0FD7804FFAE04088006A2E0CE1347
:102FF000CE13D8F802309AE555640160030230A37D
:10300000AF57EF3395E0FEEF25E0FDEE33FCAF5612
:10301000EF3395E0FEEF7805C333CE33CED8F924F5
:10302000F0F58274103EF583E5822DF582E5833C50
:10303000F583E0FAA3E0FB780CFFAE02088006A25D
:10304000E0CE13CE13D8F8540FF5587808AF03AE7E
:1030500002EF088006A2E0CE13CE13D8F8540FF585
:1030600059AF56EF3395E0FEEF7805C333CE33CE3C
:10307000D8F924F0F58274103EF583E5822DF582AF
:10308000E5833CF583E0FCA3E0FD7804FFAE040893
:103090008006A2E0CE13CE13D8F8540FF55AED54A3
:1030A0000FF55BE558700FE559700BE55A7007E5B1
:1030B0005B7003023135AD58E4FF127677AD59E409
:1030C000FF127677E55864097048855A5CAF5CFE5C
:1030D0007804EF08800633CE33CE92E0D8F8F55C62
:1030E000E55B425CE55CB4990B7D09E4FF12767701
:1030F0007D098027E55C75F00A84F55DFDE4FF122B
:103100007677E55D75F00AA4FFC3E55C9FF55DFD8C
:103110008009AD5AE4FF127677AD5BE4FF12767753
:103120007FF47E011279FA0557C3E557648094A0B5
:053130005003022F53C3
:013135002277
:025C0E008B51B8
:105C10001266CD8F52E552D394005003025CAAE580
:105C20005294334003025CAAD269AF511259FF7DEE
:105C3000527F05127677AF52124B76744F2552F58C
:105C400082E43406F583E060047D3880027D367F8F
:105C5000061276777F2C7E011279FA7F2C7E011254
:105C600079FA75F020E552A424D0F582E5F03406E7
:105C7000F583E0FEA3E0FF900000EEF0A3EFF04E0E
:105C800070077D1B7F061276777D0C7F0312767777
:105C9000900000E07002A3E06009E55214FDE4FF0B
:105CA000122F4CC269AF510259FFC268AF51127B2B
:015CB00031C2
:015CB10022D0
:026513008B51AA
:106515001266CDAD07EDD39400406BED9433506614
:10652500E4FCECFF3395E0FEEF25E0FFEE33FE756E
:10653500F020EDA424D0F582E5F03410F583E58252
:106545002FF582E5833EF583E4F0A3F00CBC10D271
:10655500749F2DF582E43406F583E4F0FCECFF33FB
:1065650095E0FE75F008EDA424F8F582E5F0340019
:10657500F583E5822FF582E5833EF583E4F00CBCD7
:0D65850008DBD2688002C268AF51127B3182
:0165920022E6
:026A84008B5134
:106A86001266CDAD07EDD394004045ED94335040EA
:106A9600E4FCECFF3395E0FEEF25E0FFEE33FE75F8
:106AA600F020EDA424D0F582E5F03406F583E582E6
:106AB6002FF582E5833EF583E4F0A3F00CBC10D2FB
:106AC600744F2DF582E43406F583E4F0D268800233
:076AD600C268AF51127B31D1
:016ADD002296
:1074A3002430F58274003EF583EDF0AF55EF33954C
:1074B300E0FEE5522FF582E5513EF583A3A3E0FFFD
:1074C300D3EF648094814008EF6480948A50012252
:0374D3007F002215
:107ADA00D3EF648094804008EF648094A15001221F
:037AEA007F0022F8
:081464008E518F528D538B5401
:10146C008F828E83A3A3A3E014F55674FC2554F548
:10147C00546403600FE55464076009E554640B6021
:10148C0003021807C3E556648094805003021807C2
:10149C00E556648094884003021807E4F555AF566E
:1014AC00EF3395E0FEEF7803C333CE33CED8F92477
:1014BC0030F58274003EF583AF55EF3395E0FEE5D1
:1014CC00822FF582E5833EF583E4F00555E555B4AE
:1014DC0008CC755504E5546403705FAF55EF339534
:1014EC00E0FEE5522FF582E5513EF583E0FFE55530
:1014FC00FD3395E0FCE5522DF582E5513CF583A3D7
:10150C00E0FD1266CD127ADAAD07AF56EF3395E0F7
:10151C00FEEF7803C333CE33CED8F91274A3AD07E4
:10152C00AF56EF3395E0FEEF7803C333CE33CED80E
:10153C00F92431F58274000217FEE5546407600348
:10154C00021639AF55EF3395E0FEE5522FF582E5E3
:10155C00513EF583E0FFE555FD3395E0FCE5522D5A
:10156C00F582E5513CF583A3E0FD1266CD127ADAE3
:10157C00AD07AF56EF3395E0FEEF7803C333CE33B0
:10158C00CED8F91274A3AD07AF56EF3395E0FEEF4A
:10159C007803C333CE33CED8F92431F58274003EB0
:1015AC00F583EDF0AF55EF3395E0FEE5522FF58264
:1015BC00E5513EF583A31274BFAD07AF56EF3395DB
:1015CC00E0FEEF7803C333CE33CED8F91266861221
:1015DC007ADAAD07AF56EF3395E0FEEF7803C333FD
:1015EC00CE33CED8F92433F58274003EF583EDF07A
:1015FC00AF55EF3395E0FEE5522FF582E5513EF500
:10160C0083E5822406F582E43583F583E0FF1274CA
:10161C00C3AD07AF56EF3395E0FEEF7803C333CE7F
:10162C0033CED8F92434F58274000217FEE55464E5
:10163C000B6003021807AF55EF3395E0FEE5522F10
:10164C00F582E5513EF583E0FFE555FD3395E0FC71
:10165C00E5522DF582E5513CF583A3E0FD1266CDF4
:10166C00127ADAAD07AF56EF3395E0FEEF7803C38D
:10167C0033CE33CED8F91274A3AD07AF56EF3395F2
:10168C00E0FEEF7803C333CE33CED8F92431F582A4
:10169C0074003EF583EDF0AF55EF3395E0FEE55267
:1016AC002FF582E5513EF583A31274BFAD07AF56FB
:1016BC00EF3395E0FEEF7803C333CE33CED8F91277
:1016CC006686127ADAAD07AF56EF3395E0FEEF7807
:1016DC0003C333CE33CED8F92433F58274003EF5F0
:1016EC0083EDF0AF55EF3395E0FEE5522FF582E533
:1016FC00513EF583E5822406F582E43583F583E0DB
:10170C00FF1274C3AD07AF56EF3395E0FEEF7803CD
:10171C00C333CE33CED8F92434F58274003EF5832E
:10172C00EDF0AF55EF3395E0FEE5522FF582E55124
:10173C003EF583E5822407F582E43583F583E0FFEB
:10174C001274C3AD07AF56EF3395E0FEEF7803C3C9
:10175C0033CE33CED8F92435F58274003EF583EDC3
:10176C00F0AF55EF3395E0FEE5522FF582E5513E93
:10177C00F583E5822408F582E43583F583E0FFE503
:10178C0055FD3395E0FCE5522DF582E5513CF58392
:10179C00E58224091266C4127ADAAD07AF56EF332C
:1017AC0095E0FEEF7803C333CE33CED8F92436F56B
:1017BC008274003EF583EDF0AF55EF3395E0FEE516
:1017CC00522FF582E5513EF583E582240AF582E439
:1017DC003583F583E0FF1274C3AD07AF56EF339535
:1017EC00E0FEEF7803C333CE33CED8F92437F5823D
:1017FC0074003EF583EDF0D2688002C268AF5312DC
:02180C007B312E
:01180E0022B7
:106FB100EF24FE601014601314601624037016D2BF
:106FC10008D2248010D209D225800AD20ED226807E
:106FD10004D20CD2277FF47E011279FA753D04E5C3
:106FE1003D70FC7F647E001279FAC224C225C2265C
:0B6FF100C227C208C209C20EC20C2257
:045652008D51AC07C3
:10565600C3EC648094815003025714EC6480948AEE
:105666004003025714E4F552AF51EF3395E0FEEFD5
:105676007803C333CE33CED8F924E8F582741A3EC4
:10568600F583AF52EF3395E0FEE5822FF582E58391
:105696003EF583E0FD74182FF582741D3EF583ED0B
:1056A600F00552E552B408C0AF04AD51127168D28C
:1056B60067AF51125AB3753D017F327E001279FAF7
:1056C600E53D70FCC267AF51125AB3E4F552E5529C
:1056D600FD3395E0FC74182DF582741D3CF583E0CE
:1056E600FBAF51EF3395E0FEEF7803C333CE33CEF5
:1056F600D8F924E8F582741A3EF583E5822DF58201
:0E570600E5833CF583EBF00552E552B408C094
:015714002272
:046E7C008D51AC0781
:106E8000D3EC64809480403CEC648094895035E479
:106E9000FDECFF3395E0FEEF7803C333CE33CED85D
:106EA000F92428F58274003EF583EDFF3395E0FE6A
:106EB000E5822FF582E5833EF583E4F00DBD08D130
:0B6EC000D2688002C268AF51127B3123
:016ECB0022A4
:04463B008C528D53BD
:10463F00D3EF648094805003024743EF64809495D6
:10464F004003024743EB648094875003024743EBD8
:10465F00648094E44003024743EF3395E0FEEF7824
:10466F0005C333CE33CED8F92460F58274033EAF41
:10467F0082F5568F57EB24FBF558D3940250030263
:10468F004743E55875F00384E5F06003024743E5BF
:10469F005875F00384F55AC394104003024743053D
:1046AF0057E557AE567002055614F5828E83E55ABC
:1046BF00F074052553F553E43552F552E4F558E5FA
:1046CF0058C3955A506A855382855283E0F559B481
:1046DF000A130557E557AE567002055614F5828E2C
:1046EF0083E4F080120557E557AE56700205561455
:1046FF00F5828E83E559F0855382855283A3E0FFBF
:10470F00855382855283A3A3E0FD1279938F5905B8
:10471F0057E557AE567002055614F5828E83E5594C
:10472F00F074032553F553E43552F5520558808F35
:0B473F00D2688002C268AF55127B31C7
:01474A00224C
:045715008F518D52D1
:10571900E551D3940050030257CCE5519415400349
:105729000257CCD269AF521259FF7D5F7F051276BD
:1057390077AD51E4FF1276777D527F041276777F39
:10574900F47E011279FA75F020E551A42460F582FE
:10575900E5F03403AF82F5558F56F583E0F55360D4
:105769004DD394004056E55394105050E55325E02D
:10577900F553755401E5532401FFE433FEC3E554A1
:105789009FEE6480F87480985032E5562554F5826E
:10579900E43555F583E0FFE5562554F582E43555A2
:1057A900F583A3E0FD1276770554055480C77D1B68
:1057B9007F061276777D5F7F05127677C269AF52D1
:0A57C9000259FFC268AF52127B3193
:0157D30022B3
:10771C008D51EFD3940A4006EFD3940F4003EF70D2
:10772C000E90063FEFF0D268AF51127B31D322C2DC
:08773C0068AF51127B31C3223A
:107744008D51EFD3940A4006EFD3940F4003EF70AA
:107754000E90063BEFF0D268AF51127B31D322C2B8
:0877640068AF51127B31C32212
:1071AE008F52E552B40B067D5F7F078034E552B4F3
:1071BE000C067D5E7F068029E552B40D067D0A7FA2
:1071CE0002801EE552B40E067D327F028013E55218
:1071DE00B40F067D467F028008E55270077D0A7F58
:0571EE00031276772278
:10761F008F51D2691259FF7D207F051276777D2E0B
:10762F007F031276777D527F0412767790063FE0C4
:0C763F00FF1271AEC269AF511259FF2258
:10764B008F51D2691259FF7D207F051276777D21EC
:10765B007F061276777D527F0412767790063BE099
:0C766B00FF1271AEC269AF511259FF222C
:1078B6008D51D3EF64809480400EEF64809486509F
:1078C60007127407D2688002C268AF51127B312258
:06732B008D51AB07AA061C
:107331008B828A83A3A3A3E0FFEB2404F582E43AC2
:107341001266C9D3EF648094804010EF648094A1E9
:10735100500990063DEFF0D2688002C268AF511229
:027361007B317E
:017363002207
:067539008D51AB07AA060C
:10753F008B828A83A3A3A3E0FFEB2404F582E43AB2
:10754F001266C9EFC39421500990063CEFF0D26840
:09755F008002C268AF51127B31B9
:017568002200
:065DF5008E518F528B530A
:105DFB00755406755540D3ED64809484407CED64F6
:105E0B008094A55075ED24FDF556D39404406BE5B5
:105E1B005620E06613F5570555E555AE547002054F
:105E2B005414F5828E83E557F074032552F552E432
:105E3B003551F551E4F556E556C395575033855218
:105E4B0082855183E0FFA3E0FD1279930555E5555B
:105E5B00AC547002055414F5828C83EFF00552E5B7
:105E6B0052700205510552E55270020551055680DC
:105E7B00C6D268AF53127B31D322C268AF53127BA9
:025E8B0031C321
:015E8D0022F2
:08474B008E518F528D538B54E7
:10475300C267D3E553648094845003024800E55351
:104763006480948D40030248008F828E83A3A3E06C
:10477300640A60030248008F828E83A3A3A3E0141C
:10478300B40800507690479675F003A4C58325F0CE
:10479300C583730247AE0247B80247C20247CC0241
:1047A30047D60247E00247EA0247F47555007556BB
:1047B30080D2678048755500755688D267803E75EC
:1047C3005500755690D2678034755500755698D24A
:1047D30067802A7555007556A0D2678020755500ED
:1047E3007556A8D26780167555007556B0D2678086
:1047F3000C755500755678D2678002C267306750D2
:10480300E4FFEF7C002556FDEC35558D82F583E4FE
:10481300F00FBF08EDE55324FB855682855583F0E1
:104823007F01E5522404F582E43551F583E5822FB7
:10483300F582E43583F583E0FEEF7C002556FDEC3D
:1048430035558D82F583EEF00FBF08D6D26880020E
:07485300C268AF54127B3173
:01485A00223B
:0461FD008E548F55D8
:106201000555E5557002055414F5828E83E0F55766
:106211006074C39408506F7F2C7E011279FAE4F503
:1062210056E556C39557505E855582855483E06087
:106231003624F5601414601714601A14601D14607C
:106241002024057028E4FD802D7D5F7F0780287D57
:106251005E7F0680227D0A7F02801C7D327F028064
:10626100167D467F0280107D0A7F03800A85558254
:10627100855483E0FDE4FF1276770555E5557002FC
:0662810005540556809B48
:0162870022F4
:022D58008B519D
:102D5A00C267EF640A6003022F33ED14B40800401F
:102D6A0003022F31902D7C75F003A4C58325F0C58D
:102D7A008373022D94022DC8022DFC022E30022EDE
:102D8A0064022E98022ECB022EFED269AF5112593E
:102D9A00FF7D577F021276777D05E4FF127677E48E
:102DAA00FDFF1276777D01E4FF1276777D527F046C
:102DBA00127677755200755380D267022F33D26923
:102DCA00AF511259FF7D577F021276777D05E4FFD6
:102DDA00127677E4FDFF1276777D02E4FF127677AA
:102DEA007D527F04127677755200755388D2670236
:102DFA002F33D269AF511259FF7D577F021276776E
:102E0A007D05E4FF127677E4FDFF1276777D03E411
:102E1A00FF1276777D527F041276777552007553CA
:102E2A0090D267022F33D269AF511259FF7D577F73
:102E3A00021276777D05E4FF127677E4FDFF1276BB
:102E4A00777D04E4FF1276777D527F0412767775D8
:102E5A005200755398D267022F33D269AF51125973
:102E6A00FF7D577F021276777D05E4FF127677E4BD
:102E7A00FDFF1276777D05E4FF1276777D527F0497
:102E8A001276777552007553A0D267022F33D26932
:102E9A00AF511259FF7D577F021276777D05E4FF05
:102EAA00127677E4FDFF1276777D06E4FF127677D5
:102EBA007D527F041276777552007553A8D26780C7
:102ECA0068D269AF511259FF7D577F021276777D1A
:102EDA0005E4FF127677E4FDFF1276777D07E4FFBB
:102EEA001276777D527F041276777552007553B049
:102EFA00D2678035D269AF511259FF7D577F0212CE
:102F0A0076777D05E4FF127677E4FDFF1276777D0A
:102F1A0008E4FF1276777D527F04127677755200A5
:102F2A00755378D2678002C267306709AF53AE52D1
:102F3A001261FD8005AF511279A5C269AF511259CC
:012F4A00FF87
:012F4B002263
:083136008E518F528D538B5412
:10313E00C2678F828E83A3A3E0640A60030231ED1F
:10314E00124A6F8E568F57D3E557943BE55694002F
:10315E0050030231E8E5579408E5569407507BC3B7
:10316E00E5536480948A5072855282855183A3A35D
:10317E00A3E0F555B40106900600023293E555B46E
:10318E000206900602023293E555B4030690060439
:10319E00023293E555B40406900606023293E555C5
:1031AE00B40506900608023293E555B4060690065D
:1031BE000A023293E555B4070690060C023293E5E7
:1031CE0055B4080690060E023293E555B4090690E2
:1031DE000610023293D26702330FD26702330F8585
:1031EE005282855183A3A3E06401600302329DAD38
:1031FE0053AF52AE51124A6F8E568F57D3E5579436
:10320E003BE5569400500302330FE5579408E556FC
:10321E009407400302330FC3E5536480948A40033E
:10322E0002330F855282855183A3A3A3E0F555B4D3
:10323E000A05900612804EE555B4010590061480DD
:10324E0044E555B40205900616803AE555B40305DB
:10325E009006188030E555B4040590061A8026E5D0
:10326E0055B4050590061C801CE555B40605900660
:10327E001E8012E555B407059006208008E555B46A
:10328E000809900622E556F0A3806FD267807285FA
:10329E005282855183A3A3E064027065AD53AF5291
:1032AE00AE51126ADE7556008F57C3E5579463E52B
:1032BE00569400504CC3E553648094885043855215
:1032CE0082855183A3A3A3E0F555B4010790063080
:1032DE00EFF0802DE555B40205900631801CE555C2
:1032EE00B403059006328012E555B40405900633FA
:1032FE008008E555B40508900634E557F08002D2F3
:0F330E0067306704C2688002D268AF54127B3107
:01331D00228D
:102655008F518D528B53E551640A6003022701E5C2
:1026650052C3940A40030228D7D269AF531259FFC7
:102675007D277F081276777D06E4FF127677E4FDE5
:10268500FF127677AD52E4FF1276777D527F041202
:102695007677E55214B4090040030228D09026B09D
:1026A50075F003A4C58325F0C583730226CB0226E6
:1026B500D10226D70226DD0226E30226E90226EF0D
:1026C5000226F50226FB900600022811900602025A
:1026D500281190060402281190060602281190067A
:1026E5000802281190060A02281190060C022811EA
:1026F50090060E022811900610022811E55164017A
:10270500600302281FE552D394004006E552940960
:102715004009E552640A600302281CD269AF5312CE
:1027250059FF7D277F081276777D06E4FF127677BD
:10273500E552B40A147D0AE4FF1276777D527F04D0
:10274500127677900612022811E552B401147D0B1A
:10275500E4FF1276777D527F041276779006140295
:102765002811E552B402147D0CE4FF1276777D52F0
:102775007F04127677900616022811E552B40313EA
:102785007D0DE4FF1276777D527F041276779006F1
:10279500188079E552B404137D0EE4FF1276777D37
:1027A500527F0412767790061A8061E552B40513BC
:1027B5007D0FE4FF1276777D527F041276779006BF
:1027C5001C8049E552B406137D10E4FF1276777D2F
:1027D500527F0412767790061E8031E552B40713B6
:1027E5007D11E4FF1276777D527F0412767790068D
:1027F500208019E552640860030228DE7D12FF126D
:1028050076777D527F04127677900622E0FEA3E06C
:10281500FF1275080228DE0228D7E551640260031D
:102825000228DEE552D3940050030228D7E55294DE
:102835000740030228D7D269AF531259FF7D277F7E
:10284500081276777D06E4FF1276777D14E4FF1291
:102855007677E55224FE60201460301460401460E1
:1028650050240470667D01E4FF1276777D527F0463
:10287500127677900630804A7D02E4FF1276777DE6
:10288500527F0412767790063180377D03E4FF127C
:1028950076777D527F0412767790063280247D0408
:1028A500E4FF1276777D527F0412767790063380A7
:1028B500117D05E4FF1276777D527F0412767790BD
:1028C5000634E0FF7E00127569800EAF531279A5BC
:1028D5008007C268AF53127B31C269AF531259FFEB
:0128E50022D0
:064A6F008E588F59A905C5
:104A75007D057C00E5592DF582E5583CF583E0C3BD
:104A8500940A400CE5592DF582E5583CF583E4F090
:104A95000DBD00010CED640A4C70D9B90610E5593D
:104AA5002405F582E43558F583E0FF7E0022E964AC
:104AB500077019E5592405F582E43558F583E07545
:104AC500F00AA4ACF0FDE55924068032E9640870CB
:104AD5003DE5592405F582E43558F583E075F06424
:104AE500A4ACF0FDE5592406F582E43558F583E0DC
:104AF50075F00AA42DFDE5F03CFCE5592407F58287
:104B0500E43558F583E02DFDE43CAF05FE22E9646C
:104B150009705AE5592405F582E43558F583E0FF17
:104B25007E007C037DE81258B2AC06AD07E559243A
:104B350006F582E43558F583E075F064A42DFDE5AE
:104B4500F03CFCE5592407F582E43558F583E0751A
:104B5500F00AA42DFDE5F03CFCE5592408F582E4B6
:104B65003558F583E02DFDE43CFEAF0522E4FEFF5C
:014B7500221D
:066ADE008E588F59A90536
:106AE4007F057E00E5592FF582E5583EF583E0C326
:106AF400940A400CE5592FF582E5583EF583E4F0FD
:106B04000FBF00010EEF64084E70D9E964077020CE
:106B1400E5592405F582E43558F583E075F00AA4B7
:106B2400FFE5592406F582E43558F583E02FFF226A
:026B34007F00E0
:016B3600223C
:104B76008F56E556D3945940147D5AE4FF12767742
:104B8600E55624A6FD7003024C77024C72E556D317
:104B9600944F401AE556945A50147D50E4FF12760D
:104BA60077E55624B0FD7003024C77024C72E55649
:104BB600D39445401AE556945050147D46E4FF12AE
:104BC6007677E55624BAFD7003024C77024C72E5FF
:104BD60056D3943B4019E556944650137D3CE4FF6A
:104BE600127677E55624C4FD7003024C77807DE586
:104BF60056D394314016E556943C50107D32E4FF6E
:104C0600127677E55624CEFD60678060E556D3942C
:104C1600274016E556943250107D28E4FF12767729
:104C2600E55624D8FD604A8043E556D3941D4016C8
:104C3600E556942850107D1EE4FF127677E556243B
:104C4600E2FD602D8026E556D394134016E5569472
:104C56001E50107D14E4FF127677E55624ECFD60B5
:104C6600108009E556C394145007AD56E4FF12763A
:024C76007722A3
:107569008E548F557C007D0A1258C4AD07E4FF1272
:1075790076777D5B7F06127677AE54AF557C007DBA
:107589000A1258C4E4FF1276777D4A7F070276779C
:047508008E548F55B9
:10750C007C007D3C1258C4124B767D057F061276AA
:10751C0077AE54AF557C007D3C1258C4ED4C600CDA
:0C752C00AF05124B767D4A7F0712767780
:017538002230
:027046008D516A
:10704800D3EF648094804038EF648094955031EF9A
:107058003395E0FEEF7805C333CE33CED8F92460FC
:10706800F58274033EAF82FEE4FD0FEFAA067001BD
:107078000E14F5828A83E4F00DBD20EED2688002FA
:07708800C268AF51127B3119
:01708F0022DE
:1072B2008F51900640E0D394024015D267125AB320
:1072C200753D037F327E001279FAE53D70FC801530
:1072D200D267AF51125AB37D1B7F061276777D0CAF
:0D72E2007F03127677C267AF51125AB322B4
:107AFF007E10900640E4F0A3DEFC7E10D268127B6D
:017B0F003144
:017B10002252
:107850008F5CD2691259FF7D607F021276777D328C
:107860007F061276777D1E7F05127677C269AF5C40
:047870001259FF2288
:1079A5008F5CD2691259FF7D607F021276777D3038
:0D79B5007F03127677C269AF5C1259FF2282
:0E7B31008F5B306803027850AF5B1279A5229B
:106686002432F58274003EF583EDF0AF55EF339575
:10669600E0FEE5522FF582E5513EF583E5822404BE
:1066A600F582E43583F583E0FFE555FD3395E0FC9F
:1066B600E5522DF582E5513CF583E5822405F58208
:0766C600E43583F583E0FDDC
:1066CD00EFD394004015EF940B5010EFC3940A5084
:1066DD0008EF75F00AA4FE8002E4FEEDD3940040AD
:1066ED000EED940B5009EDC3940A5003ED2EFEAF41
:0166FD000696
:0166FE002279
:03000000027B225E
:0F7B2200758E0078FEE4F6D8FD75816C02514B2C
:107A4900D292C0F075F008C29100A29233D291D5BA
:067A5900F0F5D0F0FF2261
:107A5F00EFC0F075F00833C291929333D291D5F005
:067A6F00F6D0F0C29122E6
:10767700EFFEEDFF1280008E2F8F30125CB2755F28
:1076870064AF5F155FEFD39400400EE4F55EE55EEF
:09769700C3943A50EC055E80F545
:0176A00022C7
:105CB200D2A885A86175A881C244853082852F83C8
:105CC200E493F560C4540FF5604360F0856080C2D0
:105CD20084D28500C2870000D287007580FF75805C
:105CE200FEC284C28500C28700000000D287007510
:105CF20080FFD24475623E756380E4F56030941D86
:105D02000560E560B464F612331EE5631563700244
:105D12001562D3E5639400E562940050DD75623E3E
:105D2200756380E4F56020941D0560E560B464F657
:105D320012331EE563156370021562D3E5639400A6
:105D4200E562940050DD8561A8C2A87F147E00122E
:025D520079FADC
:015D5400222C
:1076A1007580FDC284C28500C28700000000D287B8
:1076B100007580FF7F147E001279FA7F997E09128E
:0A76C10080008E2F8F30125CB22281
:10589000C2D530F707B2D563F0FF05F030E70CB2A0
:1058A000D5F4048463F0FF05F080018430D502F460
:0258B0000422D0
:1058B200EF8DF0A4A8F0CF8CF0A428CE8DF0A42E0A
:0258C200FE22C4
:1058C400BC000BBE0029EF8DF084FFADF022E4CCC8
:1058D400F875F008EF2FFFEE33FEEC33FCEE9DEC91
:1058E400984005FCEE9DFE0FD5F0E9E4CEFD22EDD7
:1058F400F8F5F0EE8420D21CFEADF075F008EF2F21
:10590400FFED33FD4007985006D5F0F222C398FD11
:055914000FD5F0EA22AE
:10591900EB9FF5F0EA9E42F0E99D42F0E89C45F0E4
:01592900225B
:10592A007401FF3395E0FEFDFC080808E6CF2FF668
:10593A0018E6CE3EF618E6CD3DF618E6CC3CF62241
:107B1100EFC39461400AEF947B5005EF24E0FF220C
:017B21002241
:00000001FF
